S0220000687474703A2F2F737265636F72642E736F75726365666F7267652E6E65742F1D
S12300000C9465000C94B8240C94AE240C9482000C9482000C9482000C9482000C9482003F
S12300200C9482000C9482000C9482000C944D240C9482000C947A240C94A4240C949A241F
S12300400C9412240C9482000C94C5230C9482000C946F250C9437250C9482000C94820086
S12300600C9482000C9482000C9482000C94820008000000BE922449123EABAAAA2ABECD2B
S1230080CCCC4C3E00000080BEABAAAAAA3E00000000BF000000803F0000000000084178D6
S12300A0D3BB4387D1133D190E3CC3BD4282AD2B3E68EC8276BED98FE1A93E4C80EFFFBE54
S12300C001C4FF7F3F000000000011241FBECFEFD0E1DEBFCDBF12E0A0E0B1E0EEE9FEE731
S12300E002C005900D92A831B107D9F716E0A8E1B2E001C01D92AD31B107E1F70E94850E81
S12301000C944D3F0C940000282F392FEFE3F0E0808181FDFDCF822F932F92BD81BDF89AD1
S123012080B50895282F392FEFE3F0E0808181FDFDCF1FBA822F932F92BD81BD60BD0FB682
S1230140F894FA9AF99A0FBE0895EAE7F0E0108210927C0080E880BF85EE808311B812B87D
S1230160A5E5B2E020E030E04AEF53E42D933D934D935C931397E1E3F2E084EF91E0918348
S123018080833A969183808354962D933D934D935C9313970895CF92DF92EF92FF920F935B
S12301A01F93CF93DF93282FEA01F89480919502882349F0213039F480918F02893019F079
S12301C041155105B9F580E090E0C22EDD24E090A901F090AA010091AB011091AC0124E626
S12301E030E040E050E00E94A23E6E0D7F1D801F911FCC0CDD1CCC0CDD1CF601E655FD4F93
S12302006083718382839383BE0180E090E0E080F180028113810E94A23E6E0D7F1D801F39
S1230220911F22ED32E0C20ED31EF60160837183828393837894DF91CF911F910F91FF9084
S1230240EF90DF90CF9008950F931F93CF93DF93082F10E0F801EE0FFF1FE55DFD4F8081BE
S12302609181835F93400CF05EC0F801EE0FFF1FE55DFD4F808191818F5D934014F088EDAC
S123028053C040E050E0C801880F991FDC01A55DBD4F6BE571E02D913C911197EA01CA016A
S12302A0880F991FFB01E80FF91F808191818217930798F5CA010197ABE5B1E0880F991F3A
S12302C08A0F9B1FFC0120813181F801EE0FFF1FE55DFD4F00811181FC0160817181CA0127
S12302E0880F991FA80FB91F4D915C91201B310BC901880F991F880F991F641B750B820FE2
S1230300931F0E94CD3ECE01880F991F880F991F8C0F9D1F8D97860F07C04F5F5F4F473261
S1230320510509F0B8CF86E9DF91CF911F910F9108958091F2029091F302A091F402B09134
S1230340F5020097A105B10509F057C080918F028E3161F18F3140F48A30C1F08431F1F0F7
S1230360893009F04AC00AC0803281F1803230F18832A1F1833609F040C038C088E06AE054
S123038070E04AE050E00E94CB0037C088E065E070E045E050E00E94CB002FC088E060E0F5
S12303A070E042E350E00E94CB0027C088E06EE170E04AE050E00E94CB001FC088E064E1E6
S12303C070E04AE050E00E94CB0017C088E064E170E04AE050E00E94CB000FC088E062E3EB
S12303E070E04AE050E00E94CB0007C088E064E670E04AE050E00E94CB00809133029091EB
S123040034028D549440ACF08091F6029091F702A091F802B091F9020097A105B10509F0DB
S123042071C089E06AE070E04AE550E00E94CB00089580913D0290913E0289379105ACF078
S12304408091F6029091F702A091F802B091F9020097A105B10509F055C089E06AE070E00A
S123046046E450E00E94CB00089580919F029091A002892BA1F48091F6029091F702A09102
S1230480F802B091F9020097A105B10541F089E060E070E040E050E00E94CB00089580919A
S12304A09F029091A0020197A1F48091F6029091F702A091F802B091F9020097A105B1052A
S12304C041F489E064E170E04AE050E00E94CB00089580919F029091A002029799F48091D5
S12304E0F6029091F702A091F802B091F9020097A105B10539F489E06AE070E04AE050E002
S12305000E94CB000895EF92FF920F931F9388E10FB6F89480936000109260000FBE0E94C9
S1230520F43580E091E00E94D4350F2EFFEFEF2EFFE1FF2EFCE10F2FF0E01F2FF02DD8018E
S1230540C7010197A109B109000001F0D1F7C895000060912B0270912C026353714088275A
S123056077FD8095982F0E94133D9B01AC0163E373E387EA91E40E94783C60934F017093CE
S12305805001809351019093520160914F0170915001809151019091520120E030E849E977
S12305A053E40E940C3E609353017093540180935501909356018FE491E06CE271E00E946D
S12305C0B52683E591E060E371E00E94B5262DE088E190E00FB6F894A895809360000FBE9E
S12305E020936000D801C7010197A109B109000001F0D1F7C89500001F910F91FF90EF90D3
S123060008954F925F926F927F928F929F92AF92BF92CF92DF92EF92FF920F931F937C01BC
S123062070E06B01CC0CDD1CC60ED71ECC0CDD1C86E295E0C80ED91EF601619171918080FA
S1230640918080E090E00E94113D2B013C0100E010E0C801B7010E94113D20E030E44CE9D2
S123066050E40E940C3E9B01AC0160E070E48CE995E40E94783C20E030E040E85FE30E9419
S12306800F3C9B01AC01C301B2010E94783C7B018C01AA24BB24C501B4010E94113D9B0138
S12306A0AC01C801B7010E94783C0E94CC3D7B018C01E4E0F0E0CE0EDF1EF60160817181C7
S12306C080E090E00E94113D9B01AC01C801B7010E94783C22E63BEE4BE55BE30E94103CA9
S12306E09B01AC0160E070E080E89FE30E94783C20E030E848E853E40E940F3C7B018C0168
S123070020E030E046E153E40E94C33D1816ACF0C801B70120E030E040E050E40E94743CC4
S123072088235CF0C801B70120E030E040E251E40E940C3E0E94E03C02C06CED75E0862F07
S1230740972F1F910F91FF90EF90DF90CF90BF90AF909F908F907F906F905F904F9008954E
S1230760FF920F931F93CF93DF930E940526F82E109290028823F1F0809190028F15A0F42E
S1230780CFE3D5E00091900210E00E94A125FE01E00FF11F8083809190028F5F809390023C
S12307A0809190028F1570F3609190028FE395E00E94E03310929002DF91CF911F910F9118
S12307C0FF9008952F923F924F925F926F927F928F929F92BF92CF92DF92EF92FF920F934A
S12307E01F93CF93DF93F8948091A9019091AA01A091AB01B091AC018093FA029093FB0262
S1230800A093FC02B093FD0278940F2EF1EBEF2EF1E0FF2EF02DCC24DD2400E010E00F2E06
S1230820FAEA6F2EF2E07F2EF02D0F2EF5EC4F2EF1E05F2EF02D0F2EF2ED8F2EF2E09F2E09
S1230840F02D22243324B02EE801C801880F991F880F991FF301E80FF91F80819181A28173
S1230860B3810097A105B10509F47DC0CE01880F991F880F991FF301E80FF91F2081318150
S1230880428153818091FA029091FB02A091FC02B091FD02281739074A075B0708F063C0D6
S12308A0F701A081B1819C91F201EC0FFD1F8081892B8C93CE01880F991F880F991FF3017D
S12308C0E80FF91F1082118212821382F7E0F01708F449C08CE80E94C52585E00E94C525E3
S12308E0802F0E94C52580918F0280680E94C5256091FA027091FB028091FC029091FD0289
S123090024E630E040E050E00E94F43E822F0E94C5256091FA027091FB028091FC0290913D
S1230920FD0224E630E040E050E00E94F43EBB27A52F942F832F0E94C5256091FA027091D1
S1230940FB028091FC029091FD0224E630E040E050E00E94F43ECA01AA27BB270E94C5251F
S123096083E70E94C525CE01880F991F880F991FF401E80FF91F80819181A281B38100970B
S1230980A105B10509F47EC0CE01880F991F880F991FF401E80FF91F208131814281538161
S12309A08091FA029091FB02A091FC02B091FD02281739074A075B0708F064C0F701A08132
S12309C0B1819C91F201EC0FFD1F8081809589238C93F7E0FB1508F449C08CE80E94C525DD
S12309E085E00E94C5258B2D0E94C52580918F028F770E94C5256091FA027091FB0280918E
S1230A00FC029091FD0224E630E040E050E00E94F43E822F0E94C5256091FA027091FB024E
S1230A208091FC029091FD0224E630E040E050E00E94F43EBB27A52F942F832F0E94C5258E
S1230A406091FA027091FB028091FC029091FD0224E630E040E050E00E94F43ECA01AA279E
S1230A60BB270E94C52583E70E94C525CE01880F991F880F991FF401E80FF91F1082118278
S1230A8012821382D701ED91FC919081F201EC0FFD1F80819101892311F021E030E0C90110
S1230AA002C0880F991FCA95E2F7C82AD92A0F5F1F4FE2E0F0E0EE0EFF1E0A30110509F024
S1230AC0C2CED0921F05C0921E05DF91CF911F910F91FF90EF90DF90CF90BF909F908F90EE
S1230AE07F906F905F904F903F902F9008951F9380914701813009F0A7C080911E0290917D
S1230B001F02A0912002B09121020097A105B105A9F48091A9019091AA01A091AB01B091C4
S1230B20AC0180509342A249BF4F80931E0290931F02A0932002B093210286C020911E021D
S1230B4030911F0240912002509121028091A9019091AA01A091AB01B091AC0128173907E7
S1230B604A075B0708F070C010918F028CE380938F02809133029091340290939B028093E1
S1230B809A028CE80E94C52585E00E94C52588E00E94C52580918F0280680E94C5256091C9
S1230BA0A9017091AA018091AB019091AC0124E630E040E050E00E94F43E822F0E94C525D5
S1230BC06091A9017091AA018091AB019091AC0124E630E040E050E00E94F43EBB27A52F4B
S1230BE0942F832F0E94C5256091A9017091AA018091AB019091AC0124E630E040E050E0B4
S1230C000E94F43ECA01AA27BB270E94C52583E70E94C52510938F028091A9019091AA0141
S1230C20A091AB01B091AC0180589141A94CBF4F80931E0290931F02A0932002B093210206
S1230C408091480180931D021F910895EF92FF920F931F93CF93DF93F894E090A901F09057
S1230C60AA010091AB011091AC01789440E050E0CAEAD2E062ED72E09A01CA01880F991F22
S1230C80880F991FFE01E80FF91F80819181A281B3810097A105B10531F1CA01880F991F5A
S1230CA0880F991FFE01E80FF91F80819181A281B381E816F9060A071B07A8F4CA01880F3B
S1230CC0991F880F991FFE01E80FF91F80819181A281B3818E199F09A00BB10B80839183C4
S1230CE0A283B3830CC0C901880F991F880F991FFE01E80FF91F1082118212821382C9013B
S1230D00880F991F880F991FFB01E80FF91F80819181A281B3810097A105B10531F1C901DD
S1230D20880F991F880F991FFB01E80FF91F80819181A281B381E816F9060A071B07A8F4D0
S1230D40C901880F991F880F991FFB01E80FF91F80819181A281B3818E199F09A00BB10BFC
S1230D6080839183A283B3830CC0C901880F991F880F991FFB01E80FF91F10821182128205
S1230D8013824F5F5F4F4A30510509F075CF2AEB32E0D9011D921D921D921D9282EE92E0B2
S1230DA0FC0111921192119211921D921D921D921C9213971082118212821382F90138962B
S1230DC01082118212821382FC0138961082118212821382F9013C9610821182128213828E
S1230DE0FC013C961082118212821382F90170961082118212821382FC017096108211825C
S1230E00128213822C5E3F4FF90110821182128213824496FC01108211821282138280910F
S1230E201E0290911F02A0912002B09121028E199F09A00BB10B80931E0290931F02A09335
S1230E402002B09321021092A6021092A7021092A8021092A90284E690E0A0E0B0E08093DB
S1230E608B0290938C02A0938D02B0938E020E94993B8CE80E94C52585E00E94C52589E0CB
S1230E800E94C52580918F0280680E94C525C801B70124E630E040E050E00E94F43EE22EDD
S1230EA0F32E042F152F822F0E94C525BB27A12F902F8F2D0E94C5257801002711278E2D0D
S1230EC00E94C52583E70E94C525F89484E190E0A0E0B0E08093A9019093AA01A093AB01B1
S1230EE0B093AC018093AD019093AE01A093AF01B093B0017894DF91CF911F910F91FF90D9
S1230F00EF9008950F931F93CF93DF93E1E9F3E08CEB92E09183808380E293E090931204DE
S1230F20809311049F01265F3F4F80E090E0A7EDB3E4E90188839983AA83BB83CF010296F3
S1230F400E94872B80E090E0A0EAB0E480931B0390931C03A0931D03B0931E0303E113E04A
S1230F60C8010E94872B0C5F1F4FF801108212BC11BCDF91CF911F910F9108950F931F9340
S1230F80CF93DF9302E910E084E090E06CED70E0A8010E94FA3B86E090E062E070E0A80190
S1230FA00E94FA3B88E090E063E770E0A8010E94FA3B8AE090E062E270E0A8010E94FA3B76
S1230FC08CE090E064E070E0A8010E94FA3B8EE090E06EE170E0A8010E94FA3B80E190E04F
S1230FE060E773E0A8010E94FA3B82E190E06EE170E0A8010E94FA3B84E190E068E770E06D
S1231000A8010E94FA3B86E190E068EC70E0A8010E94FA3BEFE3F0E0808181FDFDCF1FBA8B
S123102088E190E092BD81BD88E280BD0FB6F894FA9AF99A0FBEEFE3F0E0808181FDFDCF6D
S12310401FBA89E190E092BD81BD81E480BD0FB6F894FA9AF99A0FBEEFE3F0E0808181FD44
S1231060FDCF1FBA8AE190E092BD81BD81E480BD0FB6F894FA9AF99A0FBEEFE3F0E08081D5
S123108081FDFDCF1FBA8BE190E092BD81BD85E080BD0FB6F894FA9AF99A0FBEEFE3F0E037
S12310A0808181FDFDCF1FBA8CE190E092BD81BD81E480BD0FB6F894FA9AF99A0FBEEFE3E5
S12310C0F0E0808181FDFDCF1FBA8DE190E092BD81BD86E480BD0FB6F894FA9AF99A0FBEC1
S12310E002E910E08EE190E064E170E0A8010E94FA3B80E290E06EE170E0A8010E94FA3B2C
S123110082E290E068EC70E0A8010E94FA3BEFE3F0E0808181FDFDCF1FBA84E290E092BDE8
S123112081BD84E180BD0FB6F894FA9AF99A0FBEEFE3F0E0808181FDFDCF1FBA85E290E0E9
S123114092BD81BD84E180BD0FB6F894FA9AF99A0FBEEFE3F0E0808181FDFDCF1FBA86E2E9
S123116090E092BD81BD80E580BD0FB6F894FA9AF99A0FBEEFE3F0E0808181FDFDCF1FBAC1
S123118087E290E092BD81BD82E380BD0FB6F894FA9AF99A0FBEEFE3F0E0808181FDFDCF11
S12311A01FBA88E290E092BD81BD88E280BD0FB6F894FA9AF99A0FBEEFE3F0E0808181FDDE
S12311C0FDCF1FBA89E290E092BD81BD86E080BD0FB6F894FA9AF99A0FBEEFE3F0E0808173
S12311E081FDFDCF1FBA8AE290E092BD81BD10BC0FB6F894FA9AF99A0FBEEFE3F0E08081AB
S123120081FDFDCF1FBA8BE290E092BD81BD8AE080BD0FB6F894FA9AF99A0FBEEFE3F0E0AF
S1231220808181FDFDCF1FBA8CE290E092BD81BD82E180BD0FB6F894FA9AF99A0FBEEFE364
S1231240F0E0808181FDFDCF1FBA8DE290E092BD81BD8AE080BD0FB6F894FA9AF99A0FBE3E
S1231260EFE3F0E0808181FDFDCF1FBA8EE290E092BD81BD10BC0FB6F894FA9AF99A0FBE26
S1231280EFE3F0E0808181FDFDCF1FBA80E390E092BD81BD8DE280BD0FB6F894FA9AF99A00
S12312A00FBEEFE3F0E0808181FDFDCF1FBA81E390E092BD81BD83E080BD0FB6F894FA9AB1
S12312C0F99A0FBEEFE3F0E0808181FDFDCF1FBA82E390E092BD81BD81E080BD0FB6F89493
S12312E0FA9AF99A0FBEEFE3F0E0808181FDFDCF1FBA83E390E092BD81BD86E080BD0FB665
S1231300F894FA9AF99A0FBEEFE3F0E0808181FDFDCF1FBA84E390E092BD81BD86E080BD7C
S12313200FB6F894FA9AF99A0FBEEFE3F0E0808181FDFDCF1FBA85E390E092BD81BD81E0D8
S123134080BD0FB6F894FA9AF99A0FBEEFE3F0E0808181FDFDCF1FBA86E390E092BD81BDDB
S123136081E080BD0FB6F894FA9AF99A0FBEC4E6D0E002E910E0CE0168EE73E0A8010E948E
S1231380FA3BCE01029668E97AE3A8010E94FA3BCE0104966CE37FE0A8010E94FA3B2C9626
S12313A0C439D10541F727E436E0EFE3F0E0C1E4D0E0A0E4B0E0808181FDFDCF1082C9014B
S12313C00397998388831C920FB6F894FA9AF99A0FBE808181FDFDCF1082C90102979983F9
S12313E088831C920FB6F894FA9AF99A0FBE808181FDFDCF1082C9010197998388831C92D7
S12314000FB6F894FA9AF99A0FBE808181FDFDCF1082398328831C920FB6F894FA9AF99A19
S12314200FBE2C5F3F4F86E02B35380709F0C3CFEFE3F0E0808181FDFDCF1FBA80E496E092
S123144092BD81BD10BC0FB6F894FA9AF99A0FBEEFE3F0E0808181FDFDCF1FBA81E496E049
S123146092BD81BD10BC0FB6F894FA9AF99A0FBEEFE3F0E0808181FDFDCF1FBA82E496E028
S123148092BD81BD10BC0FB6F894FA9AF99A0FBEEFE3F0E0808181FDFDCF1FBA83E496E007
S12314A092BD81BD10BC0FB6F894FA9AF99A0FBEDF91CF911F910F910895CF92DF92EF927A
S12314C0FF920F931F93EFE3F0E0808181FDFDCF85E090E092BD81BDF89A80B58F3F11F43A
S12314E00E94BE07EFE3F0E0808181FDFDCF84E090E092BD81BDF89A30B5EFE3F0E0808119
S123150081FDFDCF85E090E092BD81BDF89A20B5922F80E0830F911D9093120180931101F8
S1231520EFE3F0E0808181FDFDCF86E090E092BD81BDF89A30B5EFE3F0E0808181FDFDCFF3
S123154087E090E092BD81BDF89A20B5922F80E0830F911D9C01220F331F880F991F880F55
S1231560991F880F991F280F391F3093340120933301EFE3F0E0808181FDFDCF88E090E02D
S123158092BD81BDF89A30B5EFE3F0E0808181FDFDCF89E090E092BD81BDF89A20B5922FC8
S12315A080E0830F911D9C01220F331F880F991F880F991F880F991F280F391F3093140113
S12315C020931301EFE3F0E0808181FDFDCF8AE090E092BD81BDF89A30B5EFE3F0E08081D2
S12315E081FDFDCF8BE090E092BD81BDF89A20B5922F80E0830F911D9C01220F331F880FB6
S1231600991F880F991F880F991F280F391F3093160120931501EFE3F0E0808181FDFDCF51
S12316208CE090E092BD81BDF89A30B5EFE3F0E0808181FDFDCF8DE090E092BD81BDF89ADD
S123164020B5922F80E0830F911D9C01220F331F880F991F880F991F880F991F280F391FB4
S12316603093180120931701EFE3F0E0808181FDFDCF8EE090E092BD81BDF89A30B5EFE31E
S1231680F0E0808181FDFDCF8FE090E092BD81BDF89A20B5922F80E0830F911D9C01220F29
S12316A0331F880F991F880F991F880F991F280F391F30931C0120931B01EFE3F0E0808106
S12316C081FDFDCF80E190E092BD81BDF89A30B5EFE3F0E0808181FDFDCF81E190E092BDD9
S12316E081BDF89A20B5922F80E0830F911D9093580180935701EFE3F0E0808181FDFDCF0C
S123170082E190E092BD81BDF89A30B5EFE3F0E0808181FDFDCF83E190E092BD81BDF89A0E
S123172020B5922F80E0830F911D9C01220F331F880F991F880F991F880F991F280F391FD3
S123174030931E0120931D0184EB90E09093220180932101EFE3F0E0808181FDFDCF84E126
S123176090E092BD81BDF89A30B5EFE3F0E0808181FDFDCF85E190E092BD81BDF89A20B53A
S1231780922F80E0830F911D9C01220F331F880F991F880F991F880F991F280F391F309385
S12317A0360120933501EFE3F0E0808181FDFDCF86E190E092BD81BDF89A30B5EFE3F0E09B
S12317C0808181FDFDCF87E190E092BD81BDF89A20B5922F80E0830F911D90932001809336
S12317E01F01EFE3F0E0808181FDFDCF88E190E092BD81BDF89A80B580932301EFE3F0E0D2
S1231800808181FDFDCF89E190E092BD81BDF89A80B580932401EFE3F0E0808181FDFDCF26
S12318208AE190E092BD81BDF89A80B52AE0829FC00111249093260180932501EFE3F0E02F
S1231840808181FDFDCF8BE190E092BD81BDF89A80B52AE0829FC001112490932801809389
S12318602701EFE3F0E0808181FDFDCF8CE190E092BD81BDF89A80B580932B01EFE3F0E03D
S1231880808181FDFDCF8DE190E092BD81BDF89A80B580932C01EFE3F0E0808181FDFDCF9A
S12318A08EE190E092BD81BDF89A30B5EFE3F0E0808181FDFDCF8FE190E092BD81BDF89A55
S12318C020B5922F80E0830F911D9C01220F331F880F991F880F991F880F991F280F391F32
S12318E030932E0120932D01EFE3F0E0808181FDFDCF80E290E092BD81BDF89A30B5EFE37C
S1231900F0E0808181FDFDCF81E290E092BD81BDF89A20B5922F80E0830F911D9C01220FB2
S1231920331F880F991F880F991F880F991F280F391F3093300120932F01EFE3F0E080815B
S123194081FDFDCF82E290E092BD81BDF89A30B5EFE3F0E0808181FDFDCF83E290E092BD50
S123196081BDF89A20B5922F80E0830F911D9093320180933101EFE3F0E0808181FDFDCFD5
S123198084E290E092BD81BDF89A80B52AE0829FC00111249093380180933701EFE3F0E0AF
S12319A0808181FDFDCF85E290E092BD81BDF89A80B580933901EFE3F0E0808181FDFDCF73
S12319C086E290E092BD81BDF89A80B52AE0829FC001112490933B0180933A01EFE3F0E067
S12319E0808181FDFDCF87E290E092BD81BDF89A80B52AE0829FC001112490933D018093D6
S1231A003C01EFE3F0E0808181FDFDCF88E290E092BD81BDF89A80B52AE0829FC001112449
S1231A2090933F0180933E01EFE3F0E0808181FDFDCF89E290E092BD81BDF89A80B58E5FE4
S1231A4080934001EFE3F0E0808181FDFDCF8AE290E092BD81BDF89A80B580934101EFE3EA
S1231A60F0E0808181FDFDCF8BE290E092BD81BDF89A80B52AE0829FC001112490932A01A7
S1231A80809329018091290190912A0187399105F8F084E690E090932A018093290120912A
S1231AA0290130912A01EFE3F0E0808181FDFDCF1FBA8BE290E092BD81BDC9016AE070E078
S1231AC00E94CD3E60BD0FB6F894FA9AF99A0FBEEFE3F0E0808181FDFDCF8CE290E092BDD9
S1231AE081BDF89A80B52AE0829FC00111249093430180934201EFE3F0E0808181FDFDCF12
S1231B008DE290E092BD81BDF89A80B580934401EFE3F0E0808181FDFDCF8EE290E092BD1A
S1231B2081BDF89A80B580931C02EFE3F0E0808181FDFDCF80E390E092BD81BDF89A80B557
S1231B402AE0829FC001112490934A0180934901EFE3F0E0808181FDFDCF82E390E092BD84
S1231B6081BDF89A80B580931B02EFE3F0E0808181FDFDCF83E390E092BD81BDF89A80B515
S1231B8080934601EFE3F0E0808181FDFDCF84E390E092BD81BDF89A80B52AE0829FC001E3
S1231BA0112480934501EFE3F0E0808181FDFDCF85E390E092BD81BDF89A80B5809347011F
S1231BC0EFE3F0E0808181FDFDCF86E390E092BD81BDF89A80B58093480120911101309107
S1231BE0120180911F01909120018217930788F4809111019091120120911F0130912001A2
S1231C00821B930B66E070E00E94CD3E60934B0103C089E180934B01EFE3F0E0808181FD56
S1231C20FDCF81E390E092BD81BDF89A80B540911501509116012AE0829FC001112448174D
S1231C40590788F4EFE3F0E0808181FDFDCF1FBA81E390E092BD81BD83E080BD0FB6F8948C
S1231C60FA9AF99A0FBE0F2EF4E8CF2EF0E0DF2EF02D84E690E0B6010E94C83B0F2EF6E211
S1231C80EF2EF5E0FF2EF02DF7019183808332968F0186E690E0B6010E94C83BF801918358
S1231CA0808388E690E0B6010E94C83BF7013496918380838AE690E0B6010E94C83BF701D6
S1231CC03696918380838CE690E0B6010E94C83BF7013896918380838EE690E0B6010E94C5
S1231CE0C83B2AE030E0E20EF31EF701918380830E94453A0E94CE3912BC11BC1F910F91FE
S1231D00FF90EF90DF90CF9008952F923F924F925F926F927F928F929F92AF92BF92CF928B
S1231D20DF92EF92FF920F931F93DF93CF93CDB7DEB72C970FB6F894DEBF0FBECDBFE4E508
S1231D40F0E080818093180210820F2EF1E28F2E9924F02DD4011C9204E210E0F801108264
S1231D600F2EF7E2CF2EDD24F02DD6011C920F2EFAE2EF2EFF24F02D8FEFF70180838081B9
S1231D80806880838081806480830F2EFBE2AF2EBB24F02DD5018C918F778C938C91806460
S1231DA08C930E94A8230E943E240E94A5000E941825F801808181608083808184608083A3
S1231DC0808182608083808188608083808180618083D7018C91877F8C938C918B7F8C93E8
S1231DE0F4018081806280838081806180838C9180618C938C9180628C93D5018C918F7EE4
S1231E008C93E5E2F0E080818E7F808380818D7F808380818B7F80838081877F80838081CE
S1231E208F7E8083F601808181608083E8E2F0E080818E7F8083D6018C9182608C93808111
S1231E408D7F80838C9184608C9380818B7F80838C9188608C938081877F80838C91806115
S1231E608C938C9180628C938C9180648C938C9180688C9380818F7E808380818F7D8083BC
S1231E808081806480838081806880838CE291E00E94692B60934F01709350018093510159
S1231EA09093520180E391E00E94692B609353017093540180935501909356010E948207F1
S1231EC00E945D0A7894EAE2F0E080818260808380818E7F80830E946C378AEA0E94C52511
S1231EE081E00E94C525809118020E94C52585E50E94C52582E08093230260914F01709168
S1231F00500180915101909152012DEC3CEC4CEC5EE30E94743C882384F460914F01709124
S1231F20500180915101909152012FE832EC45EF5CE30E94C33D1816C4F087E19FE9A2E0D7
S1231F40BDE380934F0190935001A0935101B093520180E090ECACE1B1E480935301909363
S1231F605401A0935501B093560189E060E070E045E050E00E94CB0010921E0210921F02A5
S1231F801092200210922102E6EAF2E0108211821282138234971082118212821382109209
S1231FA09C021092A00210929F020F2EF4E8CF2EF0E0DF2EF02D84E690E0B6010E94C83BB2
S1231FC00F2EF6E2EF2EF5E0FF2EF02DF7019183808332968F0186E690E0B6010E94C83B0D
S1231FE0D80111969C938E9388E690E0B6010E94C83BF70134969183808380E790E0B6016C
S12320000E94C83BF70136969183808382E790E0B6010E94C83BF70138969183808384E7BF
S123202090E0B6010E94C83BEAE0F0E0EE0EFF1ED70111969C938E93A8952DE088E190E02B
S12320400FB6F894A895809360000FBE20936000E3E3F2E03C96FA83E9830F2EF6ED4F2EAB
S1232060F2E05F2EF02D0F2EF2EA2F2EF2E03F2EF02D91012C5F3F4F3C832B838BE392E016
S123208008969E838D83A1E3B2E05096B887AF83E7E2F4E03296FA87E9872BE232E0285F04
S12320A03F4F3C872B8795B1E8E2F0E0990F947080818B7F892B8083908192959695977061
S12320C0927080818D7F892B8083A8958091A9019091AA01A091AB01B091AC018158934CEF
S12320E0A94CB14010F00E9426060E94AF3A8091A9019091AA01A091AB01B091AC0120919A
S1232100AD013091AE014091AF015091B001821B930BA40BB50B89589341A040B040F0F07B
S12321208091A9019091AA01A091AB01B091AC018093AD019093AE01A093AF01B093B001DF
S123214080918F02843151F4A3E3B2E08D919C91E981FA81608171810E946739F20180818E
S12321609181A281B3810097A105B10509F0BCC080914101882311F04B990AC0AFE3B2E0B9
S12321802D913C918091390190E0281739073CF5809196029091970201969093970280937C
S12321A096028091960290919702885B984808F49BC080919502882309F096C081E060E0C3
S12321C070E040E050E00E94CB0081E08093950288EB98E8909397028093960285C0809133
S12321E09602909197020197909397028093960280919602909197020B9708F075C0809147
S12322009502813009F070C0109295028AE090E0909397028093960280918F028E31B9F5C0
S12322206091A9017091AA018091AB019091AC01E0901D01F0901E01A0901D01B0901E01EE
S123224060901D0170901E0124E630E040E050E00E94F43E00E010E02E0D3F1D401F511FD9
S12322602C5E3F4F4F4F5F4FCC24DD242A0D3B1D4C1D5D1D88249924260D371D481D591DC8
S1232280E6EAF2E020833183428353832DC06091A9017091AA018091AB019091AC01E09077
S12322A01D01F0901E01A0901D01B0901E0124E630E040E050E00E94F43E00E010E02E0D67
S12322C03F1D401F511F2C5E3F4F4F4F5F4FCC24DD242A0D3B1D4C1D5D1DA6EAB2E02D9326
S12322E03D934D935C9313970E94990180918F028E3111F40C94BC198F31A0F48A3009F46F
S1232300B8C48B3038F4882359F1893011F00C947120CEC0833109F4F6C6843111F00C9425
S1232320712015C7883211F40C94001E893250F48F3111F40C940A1B803211F00C94712042
S12323400C946F1B8D3311F40C94271F833611F40C9411208C3311F00C9471200C94B81EAE
S123236084E18093590180935A01E8E2F0E080818E7F808380818D7F808380919C02882304
S123238051F480919F029091A002892B21F01092A00210929F028091A9019091AA01A0917B
S12323A0AB01B091AC0189589341A040B04010F40C94732010929E0210929D0280E060E0A0
S12323C070E04AE050E00E94CB00A1E4B2E02D913C9180912501909126012817390760F0F2
S12323E088E280938F0280912401809359018091240180935A0154C0E3E3F2E080819181C5
S1232400883C9105A4F088E280938F028FE090E09093920280939102109293028091240113
S1232420809359018091240180935A0139C0A3E3B2E08D919C91119787399105C4F0809168
S12324402401809359018091240180935A0189E080938F0210929202109291028D919C917F
S123246090939902809398021092930219C080912401809359018091240180935A0189E02D
S123248080938F02109292021092910210929302E3E3F2E0808191819093990280939802DC
S12324A0D1011D921D921D921C9213970C94732010921E0210921F021092200210922102A0
S12324C0EAEDF2E020813181428153818091A9019091AA01A091AB01B091AC0188519C4F4F
S12324E0AF4FBF4F281739074A075B07B0F4F10180819181A281B3810297A105B10568F04D
S1232500A3E3B2E08D919C9145973CF082E060E070E048EE53E00E94CB00EEEDF2E08081D6
S12325209181A281B3810097A105B10509F074C08091910290919202889708F06DC0809160
S12325402401809359018091240180935A014091190250911A0283E060E070E00E94CB00F8
S123256080919C028F5F80939C0280919102909192028A96909392028093910280913A01E7
S123258090913B0190931A018093190180919C028230A8F0EFE3F0E0808181FDFDCF81E325
S12325A090E092BD81BDF89A40B58AE0489FA001112481E060E070E00E94CB0009C0409174
S12325C015015091160181E060E070E00E94CB00F10180819181A281B3810196A11DB11D0C
S12325E080839183A283B3836091A9017091AA018091AB019091AC0124E630E040E050E029
S12326000E94F43E822F932FA42FB52FEB81FC8180839183A283B383EEEDF2E0808191819D
S1232620A281B3810097A105B10509F070C0F10180819181A281B3810197A105B10509F0DA
S123264066C0F20180819181A281B3810097A105B10509F05CC0A3E3B2E08D919C91909365
S1232660990280939802409113015091140183E060E070E00E94CB00809113019091140178
S123268020919102309192026AE070E00E94CD3E620F731F709392026093910284E060E092
S12326A070E040EB54E00E94CB0081E090E090939E0280939D02F10180819181A281B38158
S12326C00196A11DB11D80839183A283B3836091A9017091AA018091AB019091AC0124E685
S12326E030E040E050E00E94F43E822F932FA42FB52FEB81FC8180839183A283B38380910C
S12327002401809359018091240180935A018091980290919902A3E3B2E02D913C9144969B
S123272028173907E0F088EE93E09093990280939802809124012091230190E0820F911D38
S12327409595879580935901809124012091230190E0820F911D9595879580935A01EEED79
S1232760F2E080819181A281B3810097A105B105A1F5F10180819181A281B3810297A105F5
S1232780B10558F180911C0290E00496880F991FEBE2F2E0E80FF91F408151818091420119
S12327A09091430120914401821B910948175907A0F480911B02813039F480E060E070E034
S12327C044E150E00E94CB00409113015091140183E064E170E00E94CB00A2EEB2E02D9113
S12327E03D914D915C918091A9019091AA01A091AB01B091AC0188519C4FAF4FBF4F2817DB
S123280039074A075B07B0F480919D0290919E02059780F484E060E070E040EB54E00E94A7
S1232820CB0080919D0290919E02019690939E0280939D02E2EEF2E080819181A281B38140
S12328400097A105B105C1F4A3E3B2E02D913C9180912101909122018217930768F484E0BF
S123286060E070E048EB5BE00E94CB008AE090E090939E0280939D02F10180819181A28172
S1232880B3810297A105B10508F4CFC020813181428153818091400190E0A0E0B0E0281785
S12328A039074A075B0708F0C0C0F20180819181A281B3810097A105B10509F0B6C0A3E364
S12328C0B2E0ED90FC90F101608171818281938100912101109122010253104029E130E047
S12328E040E050E00E94A23E060F171F0E151F0508F09BC06091A9017091AA018091AB0119
S12329009091AC01A6EAB2E0ED90FD900D911C9124E630E040E050E00E94F43E2E193F09A1
S1232920400B510B233331054105510508F47DC06091A9017091AA018091AB019091AC01B9
S1232940E6EAF2E0E080F1800281138124E630E040E050E00E94F43EE216F3060407150793
S123296008F063C0AFE3B2E02D913C9180915701909158012817390708F057C084E060E074
S123298070E040E157E20E94CB006091190170911A01409117015091180181E00E94CB0044
S12329A0F10180819181A281B3810196A11DB11D80839183A283B3836091A9017091AA01DB
S12329C08091AB019091AC01E0901901F0901A01A0901701B090180100E010E024E630E0B8
S12329E040E050E00E94F43EE20EF31E041F151FCC24DD24EA0CFB1C0C1D1D1DAB81BC818D
S1232A00ED92FD920D931C931397809137019091380190931A018093190180912301809355
S1232A2059018091230180935A01F10120813181428153818091400190E0A0E0B0E02817A8
S1232A4039074A075B0708F462C0F20180819181A281B3810097A105B10509F058C0A3E37A
S1232A60B2E02D913C9180913C0190913D0182179307E0F4EFE3F2E0208131818091570121
S1232A80909158012817390788F4D1011D921D921D921C9213978AE080938F0282E060E0D6
S1232AA070E040ED57E00E94CB0031C06091A9017091AA018091AB019091AC01E6EAF2E08C
S1232AC0E080F1800281138124E630E040E050E00E94F43E80EB94E0A0E0B0E0E80EF91ED0
S1232AE00A1F1B1FE216F3060407150780F4D1011D921D921D921C9213978AE080938F029E
S1232B0082E060E070E04AE050E00E94CB00EEEDF2E080819181A281B3810097A105B105EE
S1232B20D1F080911C0290E00496880F991FEBE2F2E0E80FF91F20813181809142019091D2
S1232B4043018217930738F483E060E070E040E050E00E94CB00EEEDF2E080819181A2813B
S1232B60B3810097A105B10549F5F10180819181A281B3810297A105B10500F180911C027B
S1232B8090E00496880F991FEBE2F2E0E80FF91F40815181809142019091430120914401E8
S1232BA0821B91094817590748F4409113015091140183E060E070E00E94CB00F1018081B1
S1232BC09181A281B3810297A105B10570F1E2EEF2E080819181A281B3810097A105B10533
S1232BE021F580919D0290919E020597F0F0A3E3B2E08D919C91883C9105BCF480919C02B2
S1232C00823048F410928F0281E090E09093A00280939F020AC084E060E070E048E853E123
S1232C200E94CB0083E680938F02E1E4F2E02081318180912501909126018C599F4F28179B
S1232C40390710F40C94732088E280938F02A3E3B2E08D919C91909399028093980280910C
S1232C6098029091990290939B0280939A020C94732010921E0210921F021092200210926D
S1232C802102A8951092A00210929F0210929C02EEEDF2E080819181A281B3810097A105B5
S1232CA0B105D1F080911C0290E00496880F991FEBE2F2E0E80FF91F2081318180914201BC
S1232CC0909143018217930738F483E060E070E040E050E00E94CB00AAEDB2E02D913D91C7
S1232CE04D915C918091A9019091AA01A091AB01B091AC0188519C4FAF4FBF4F2817390764
S1232D004A075B0780F4F10180819181A281B3810097A105B10539F482E060E070E040EDED
S1232D2057E00E94CB00E2EDF2E080819181A281B3810097A105B105A1F4F1018081918153
S1232D40A281B3810097A105B10559F06091350170913601409133015091340180E00E9460
S1232D60CB008091230180935A018091230180935901A2EEB2E02D913D914D915C918091B5
S1232D80A9019091AA01A091AB01B091AC0188519C4FAF4FBF4F281739074A075B0738F4C0
S1232DA084E060E070E048EE53E00E94CB00F20180819181A281B3810097A105B10509F0FC
S1232DC0AFC0F10180819181A281B3810097A105B10509F0A5C06091A9017091AA0180917B
S1232DE0AB019091AC01A6EAB2E0ED90FD900D911C9124E630E040E050E00E94F43EE216A8
S1232E00F3060407150708F08BC06091A9017091AA018091AB019091AC01E6EAF2E0A080B7
S1232E20B180C280D380E0903E01F0903F0124E630E040E050E00E94F43E2A193B094C093F
S1232E405D0900E010E0E216F3060407150708F067C0A3E3B2E0AD90BC90E0901F01F09050
S1232E60200160914B01F1012081318142815381CC24B7FCC094DC2C70E080E090E00E9453
S1232E80A23E00E010E06E0D7F1D801F911F6A157B058C059D0508F000C1AFE3B2E02D914B
S1232EA03C9180915701909158012817390708F0F4C040911B0150911C0181E060E070E057
S1232EC00E94CB004091490150914A0182E060E070E00E94CB00F10180819181A281B3817F
S1232EE00196A11DB11D80839183A283B3836091A9017091AA018091AB019091AC0124E65D
S1232F0030E040E050E00E94F43E822F932FA42FB52FEB81FC8180839183A283B383BDC077
S1232F20F20180819181A281B3810097A105B10509F0B3C0F10180819181A281B3810097DE
S1232F40A105B10509F4A9C06091A9017091AA018091AB019091AC01A6EAB2E0ED90FD90AD
S1232F600D911C9124E630E040E050E00E94F43EE216F3060407150708F08FC06091A901CA
S1232F807091AA018091AB019091AC01E6EAF2E0A080B180C280D38080901D0190901E0101
S1232FA0E0901B01F0901C0124E630E040E050E00E94F43E2A193B094C095D09E80CF91C5B
S1232FC000E010E0E216F3060407150708F065C0A3E3B2E0AD90BC90E0901F01F090200116
S1232FE060914B01F1012081318142815381CC24B7FCC094DC2C70E080E090E00E94A23E13
S123300000E010E06E0D7F1D801F911F6A157B058C059D0508F041C0AFE3B2E02D913C919C
S1233020809157019091580128173907B0F540911B0150911C0181E060E070E00E94CB003C
S12330404091490150914A0182E060E070E00E94CB00F10180819181A281B3810196A11D15
S1233060B11D80839183A283B3836091A9017091AA018091AB019091AC0124E630E040E000
S123308050E00E94F43E822F932FA42FB52FEB81FC8180839183A283B383F101808191819E
S12330A0A281B3810297A105B10518F083E180938F02A3E3B2E08D919C918436910514F4F5
S12330C010928F02E1E4F2E02081318180912501909126012817390710F40C9473208EE12B
S12330E080938F02A3E3B2E08D919C919093990280939802809198029091990290939B0233
S123310080939A02F0C784E180938F02F10110821182128213820E945D0AE8E2F0E0808158
S123312081608083808182608083109292021092910210929C0210921E0210921F021092EF
S12331402002109221028081877F8083CCC78091230180935A0180912301809359010E9400
S12331607705E2EDF2E080819181A281B3810097A105B10559F46091350170913601409154
S123318033015091340180E00E94CB00A2EEB2E02D913D914D915C918091A9019091AA0114
S12331A0A091AB01B091AC0188519C4FAF4FBF4F281739074A075B0738F484E060E070E01E
S12331C040EB54E00E94CB00F20180819181A281B3810097A105B10509F0B2C06091A901C9
S12331E07091AA018091AB019091AC01A6EAB2E0ED90FD900D911C9124E630E040E050E0B3
S12332000E94F43EE216F3060407150708F098C06091A9017091AA018091AB019091AC019C
S1233220E6EAF2E0A080B180C280D38080901D0190901E01E0901B01F0901C0124E630E052
S123324040E050E00E94F43E2A193B094C095D09E80CF91C00E010E0E216F3060407150713
S12332600CF06EC0A7E2B4E02D913C9180911101909112018217930708F062C0EFE3F2E030
S12332802081318180915701909158012817390708F056C080911D02882331F080911D023B
S12332A0815080931D0209C040911B0150911C0181E060E070E00E94CB00A3E3B2E08D91BF
S12332C09C919093990280939802809194028F5F80939402F10180819181A281B381019621
S12332E0A11DB11D80839183A283B3836091A9017091AA018091AB019091AC0124E630E0E0
S123330040E050E00E94F43E822F932FA42FB52FEB81FC8180839183A283B38340914901E5
S123332050914A0182E060E070E00E94CB008091A102813029F48EE180938F021092A10224
S1233340A1E4B2E02D913C9180912501909126012817390720F081E08093A10202C010923E
S1233360A102E3E3F2E080819181843691050CF0BAC610928F02B7C610921E0210921F02FA
S12333801092200210922102A3E3B2E02D913C91119780919A0290919B028217930730F493
S12333A08D919C9190939B0280939A0210929C0280912B018093590180912B0180935A01BA
S12333C080919A0290919B028752924038F0E3E3F2E080819181C2970CF4D6C0A2EEB2E0EF
S12333E02D913D914D915C918091A9019091AA01A091AB01B091AC0188519C4FAF4FBF4F50
S1233400281739074A075B0738F484E060E070E040EB54E00E94CB00E2EDF2E080819181D6
S1233420A281B3810097A105B10559F46091350170913601409133015091340180E00E9475
S1233440CB00F20180819181A281B3810097A105B10509F099C06091A9017091AA018091A3
S1233460AB019091AC01A6EAB2E0ED90FD900D911C9124E630E040E050E00E94F43EE21621
S1233480F3060407150708F07FC06091A9017091AA018091AB019091AC01E6EAF2E0A0803D
S12334A0B180C280D38080902F0190903001E0902D01F0902E0124E630E040E050E00E9458
S12334C0F43E2A193B094C095D09E80CF91C00E010E0E216F306040715070CF055C0A7E2E9
S12334E0B4E02D913C9180913101909132018217930708F049C0EFE3F2E0208131818091D6
S123350057019091580128173907F0F540912D0150912E0181E060E070E00E94CB00409133
S1233520490150914A0182E060E070E00E94CB00A3E3B2E08D919C919093990280939802E4
S1233540F10180819181A281B3810196A11DB11D80839183A283B3836091A9017091AA012F
S12335608091AB019091AC0124E630E040E050E00E94F43E822F932FA42FB52FEB81FC816B
S123358080839183A283B383A1E4B2E08D919C912091250130912601409127015091280191
S12335A0241B350B82179307F8F4E3E3F2E080819181803991051CF410928F0215C0D10185
S12335C01D921D921D921C92139780E280938F021092990210929802809124018093590160
S12335E08091240180935A01E1E4F2E04081518120912501309126018091290190912A01B3
S1233600820F931F8417950708F06DC588E280938F0269C580912B018093590180912B01DF
S123362080935A01AAEDB2E02D913D914D915C918091A9019091AA01A091AB01B091AC0146
S123364088519C4FAF4FBF4F281739074A075B0738F482E060E070E048E552E00E94CB007A
S1233660E2EEF2E020813181428153818091A9019091AA01A091AB01B091AC0188519C4FA4
S1233680AF4FBF4F281739074A075B0738F484E060E070E040EB54E00E94CB006091A90161
S12336A07091AA018091AB019091AC01E0908B02F0908C0200918D0210918E0224E630E059
S12336C040E050E00E94F43EE216F3060407150708F009C510928F0210929C0204C5AAED11
S12336E0B2E02D913D914D915C918091A9019091AA01A091AB01B091AC0188519C4FAF4FC9
S1233700BF4F281739074A075B0760F4F10180819181A281B38182E060E070E040ED57E05F
S12337200E94CB00A2EEB2E02D913D914D915C918091A9019091AA01A091AB01B091AC014D
S123374088519C4FAF4FBF4F281739074A075B0738F484E060E070E040EB54E00E94CB0077
S1233760F10180819181A281B3810097A105B10509F081C0F20180819181A281B3810097C8
S1233780A105B10509F077C0409113015091140183E060E070E00E94CB004091450181E0E6
S12337A06CE370E050E00E94CB00F10180819181A281B3810196A11DB11D80839183A2830E
S12337C0B3836091A9017091AA018091AB019091AC01E0901D01F0901E0124E630E040E076
S12337E050E00E94F43E89019A01C70165E070E00E94CD3E660F771F660F771F80E090E0AC
S1233800601771078207930758F56091A9017091AA018091AB019091AC01E0901D01F09065
S12338201E0124E630E040E050E00E94F43E89019A01C70165E070E00E94CD3E660F771FED
S1233840660F771F80E090E0061B170B280B390BA6EAB2E00D931D932D933C9313972BC039
S123386082E390E0A0E0B0E0E6EAF2E080839183A283B38320C0F10180819181A281B3810F
S12338800197A105B105B9F4F20180819181A281B3810097A105B10571F480919802909102
S12338A09902892B41F4A3E3B2E08D919C919093990280939802E3E3F2E0208131818091B6
S12338C09802909199028C599F4F28173907F0F48091980290919902892BC1F08081918179
S12338E0805991409CF4EEEDF2E080819181A281B3810097A105B10549F44091130150917D
S1233900140183E060E070E00E94CB00EEEDF2E080819181A281B3810097A105B10571F0C3
S1233920A3E3B2E08D919C91875292403CF083E060E070E040E050E00E94CB00E3E3F2E001
S12339402081318180919802909199028C599F4F8217930730F48091980290919902892B64
S123396041F4A3E3B2E08D919C91875292400CF4F3C0EEEDF2E080819181A281B38100979F
S1233980A105B10539F083E060E070E040E050E00E94CB0084E690E09093990280939802A9
S12339A080912301809359018091230180935A01F10180819181A281B3810097A105B1056F
S12339C009F4CAC020813181428153818091460190E00296AA2797FDA095BA2F2817390710
S12339E04A075B0708F0B8C0F20180819181A281B3810097A105B10509F0AEC0A3E3B2E0D1
S1233A00ED90FC90F101608171818281938100912101109122010951104029E130E040E062
S1233A2050E00E94A23E060F171F0E151F0508F093C06091A9017091AA018091AB019091CE
S1233A40AC01A6EAB2E0ED90FD900D911C9124E630E040E050E00E94F43E2E193F09400B26
S1233A60510B233331054105510508F475C06091A9017091AA018091AB019091AC01E6EAEB
S1233A80F2E0E080F1800281138124E630E040E050E00E94F43EE216F3060407150708F01A
S1233AA05BC0AFE3B2E02D913C9180915701909158012817390708F04FC084E060E070E0DB
S1233AC040E157E20E94CB006091190170911A01409117015091180181E00E94CB00F10151
S1233AE080819181A281B3810196A11DB11D80839183A283B3836091A9017091AA0180916B
S1233B00AB019091AC01E0901901F0901A01A0901701B090180100E010E024E630E040E057
S1233B2050E00E94F43EE20EF31E041F151FCC24DD24EA0CFB1C0C1D1D1DAB81BC81ED92DC
S1233B40FD920D931C931397809137019091380190931A0180931901F101208131814281C3
S1233B6053818091400190E0A0E0B0E0281739074A075B0750F1F20180819181A281B381CB
S1233B800097A105B10509F5A3E3B2E02D913C9180913C0190913D0182179307B0F4F10117
S1233BA010821182128213828AE080938F02EB81FC8180819181A281B38180559040A040CD
S1233BC0B04080839183A283B383A3E3B2E08D919C918436910524F410929C0210928F0241
S1233BE0E1E4F2E02081318180912501909126018217930708F077C28EE180938F0273C2AC
S1233C0010921E0210921F02109220021092210280912C018093590180912C0180935A013B
S1233C20F20180819181A281B3810097A105B10539F081E060E070E040E050E00E94CB0059
S1233C40A3E3B2E08D919C918059914044F080912301809359018091230180935A01E3E314
S1233C60F2E080819181883C91050CF46AC0A2EEB2E02D913D914D915C918091A901909182
S1233C80AA01A091AB01B091AC0188519C4FAF4FBF4F281739074A075B0738F484E060E0D8
S1233CA070E040EB54E00E94CB00E2EDF2E080819181A281B3810097A105B10591F4809150
S1233CC03501909136014091330150913401BC01660F771F680F791F7695679580E00E9457
S1233CE0CB00A1E4B2E08D919C9120912501309126014091270150912801241B350B8217B9
S1233D00930708F0F0C1E3E3F2E080819181805991400CF0E8C1D1011D921D921D921C92D5
S1233D20139780E280938F02109299021092980280912401809359018091240180935A010F
S1233D40D2C1E1E4F2E08081918120912501309126014091270150912801241B350B821748
S1233D60930708F0C0C110928F0210929C02BBC18091230180935A018091230180935901F8
S1233D80E2EDF2E080819181A281B3810097A105B10559F460913501709136014091330170
S1233DA05091340180E00E94CB00A2EEB2E02D913D914D915C918091A9019091AA01A091EB
S1233DC0AB01B091AC0188519C4FAF4FBF4F281739074A075B0738F484E060E070E040EBF8
S1233DE054E00E94CB00E3E3F2E02081318180919A0290919B028217930730F4808191815E
S1233E0090939B0280939A02A3E3B2E02D913C91119780919A0290919B028659904028178B
S1233E20390728F08D919C918F5E92402CF0109294028DE380938F02E3E3F2E08081918109
S1233E40843691050CF04FC110928F024CC1E2EDF2E080819181A281B3810097A105B105C4
S1233E6059F46091350170913601409133015091340180E00E94CB00A2EEB2E02D913D91FC
S1233E804D915C918091A9019091AA01A091AB01B091AC0188519C4FAF4FBF4F28173907B2
S1233EA04A075B0738F484E060E070E040EB54E00E94CB00F20180819181A281B38100976B
S1233EC0A105B10509F08BC06091A9017091AA018091AB019091AC01A6EAB2E0ED90FD9040
S1233EE00D911C9124E630E040E050E00E94F43EE216F3060407150708F071C06091A90159
S1233F007091AA018091AB019091AC01E6EAF2E0A080B180C280D380E0901D01F0901E01B1
S1233F2080901B0190901C0124E630E040E050E00E94F43E2A193B094C095D09EE0CFF1C7F
S1233F40E80CF91C00E010E0E216F3060407150708F045C0A3E3B2E02D913C9180911101A9
S1233F609091120182179307D0F540911B0150911C0181E060E070E00E94CB00E3E3F2E030
S1233F80808191819093990280939802809194028F5F80939402F10180819181A281B38105
S1233FA00196A11DB11D80839183A283B3836091A9017091AA018091AB019091AC0124E68C
S1233FC030E040E050E00E94F43E822F932FA42FB52FEB81FC8180839183A283B383809113
S1233FE09402843028F01092940283E180938F02A1E4B2E02D913C918091250190912601FA
S12340008217930718F48EE180938F02E3E3F2E080819181843691050CF065C010928F02FB
S123402062C080912401809359018091240180935A01EEEDF2E080819181A281B381009765
S1234040A105B10539F083E060E070E040E050E00E94CB00F20180819181A281B381009733
S1234060A105B10539F081E060E070E040E050E00E94CB00EAEDF2E080819181A281B381F6
S12340800097A105B10539F082E060E070E040E050E00E94CB00E2EDF2E080819181A2817A
S12340A0B3810097A105B10539F080E060E070E040E050E00E94CB00439907C084E060E0B8
S12340C070E040EB54E00E94CB0082E090E09093A00280939F02E8E2F0E0808188608083EF
S12340E002C010928F0280910203883398F01092020383E193E00E94FF2683E993E00E94A8
S1234100FF268091FE029091FF0201969093FF028093FE02A8950E94A137882309F46DC0E9
S123412080918F024091A9015091AA016091AB017091AC012BE232E00E94B83781E0809363
S12341402302AB85BC856D917C91882777FD8095982F0E94133D6093CB037093CC03809323
S1234160CD039093CE0380917C008630F1F40E94B3378823D1F0809178009091790060E0F4
S12341800E9401036AE070E00E94E13E862F972FEDE2F2E091838083808191818B3591057E
S12341A03CF083E680938F0203C086E080937C00E3E3F2E080819181A7E2B4E011969C936C
S12341C08E93E985FA85208131818D919C911197820F931F9695879591838083FD0134961E
S12341E020813181A985BA858D919C91820F931F9695879591838083A5C2809124028130C0
S123420009F0A0C21092240280912302843009F07DC00F2EF9E58F2EF2E09F2EF02DF401CE
S12342206081718182819381E0907800F090790026E636E646E65FE30E940C3E5B016C0164
S123424000E010E0C801B7010E94113D20E932EC45EF5DE30E940C3E9B01AC01C601B501CC
S12342600E94103CD4016D937D938D939C9313976D917D918D919C910E94E03CE3E3F2E0C1
S12342807183608380819181A7E2B4E011969C938E93E985FA85208131818D919C911197E9
S12342A0820F931F9695879591838083FD01349620813181A985BA858D919C91820F931F43
S12342C0969587959183808311E01093230210932302E3E3F2E060817181882777FD809558
S12342E0982F0E94133D6093CB037093CC038093CD039093CE03E2E2F0E080818F7D8083F3
S123430080818F7E808310937C001CC280912302813041F486E0809323020E94AF3A1092A4
S12343207C0010C280912302853009F046C00F2EFDE58F2EF2E09F2EF02DD4016D917D91C8
S12343408D919C91E0907800F09079002DEC3CEC4CE45FE30E940C3E5B016C0100E010E0F5
S1234360C801B7010E94113D20E932EC45E75EE30E940C3E9B01AC01C601B5010E94103C94
S1234380F401608371838283938360817181828193810E94E53C709336026093350292E0AE
S12343A090932302E2E2F0E080818062808380818061808390937C00C5C180912302823045
S12343C019F5AFE3B2E02D913C9111974091780050917900C901880F991F880F991F880FD2
S12343E0991F821B930B840F951F96958795969587959695879511969C938E9387E0809339
S1234400230210927C009EC180912302863071F410922302E2E2F0E0808180628083808163
S12344208F7E808383E080937C008CC180912302882309F085C00F2EF9E48F2EF2E09F2E94
S1234440F02DF4016081718182819381E0907800F090790023E333E343E75FE30E940C3E07
S12344605B016C0100E010E0C801B7010E94113D2DEC3CEC4CE45DE30E940C3E9B01AC0148
S1234480C601B5010E94103CD4016D937D938D939C9313976D917D918D919C910E94E53CB5
S12344A0EBE2F2E07183608385E08093230260817181E0904F01F0905001009151011091FD
S12344C05201882777FD8095982F0E94133DA80197010E940C3E609385027093860280934F
S12344E0870290938802609185027091860280918702909188022091530130915401409150
S12345005501509156010E940F3C6093850270938602809387029093880280918502909115
S12345208602A0918702B091880280934B0390934C03A0934D03B0934E0310927C0002C19F
S123454080912302873009F043C0A5E6B2E06D917D918D919C91E0907800F090790026E60D
S123456036E646E65FE30E940C3E5B016C0100E010E0C801B7010E94113D20E932EC45EF5C
S12345805DE30E940C3E9B01AC01C601B5010E94103CE5E6F2E060837183828393836081C7
S12345A07181828193810E94E03C70933A026093390283E080932302E2E2F0E080818F7D87
S12345C0808380818061808386E080937C00BAC080912302833009F052C0A5E5B2E06D9172
S12345E07D918D919C91E0907800F090790026E636E646E65FE30E940C3E5B016C0100E052
S123460010E0C801B7010E94113D2DEC3CEC4CEC5DE30E940C3E9B01AC01C601B5010E9428
S1234620103CE5E5F2E0608371838283938360817181828193810E94E53CA1E3B2E0119632
S12346407C936E9388E0809323028D919C9160E00E940103EF81F88591838083808191815E
S12346606AE070E00E94E13E862F972FE1E3F2E03C969183808387E080937C0063C08091B7
S12346802302883009F058C0A9E6B2E06D917D918D919C910F2EF8E78F2E9924F02DF40108
S12346A0E080F1802DEC3CEC4CE45FE30E940C3E5B016C0100E010E0C801B7010E94113D7C
S12346C02DEC3CEC4CE45EE30E940C3E9B01AC01C601B5010E94103CA9E6B2E06D937D9353
S12346E08D939C931397EBE3F2E020813181D4014D915C91C901880F991F880F991F880F2B
S1234700991F821B930B840F951F9695879596958795969587959183808384E080932302D3
S12347208081918161E00E940103ED81FE819183808310927C0006C0109223028091230296
S123474080937C000E94E2030E94B0030C945310E5E4F0E01082AEE6B0E08C9183608C9379
S123476080818360808317BCEAE2F0E0808180618083808180628083EBE2F0E080818F7E69
S1234780808380818F7D808308951F920F920FB60F9211245F936F937F938F939F93AF93DC
S12347A0BF93EF93FF93F894EBE2F0E0808180618083808180628083809101038F5F809385
S12347C00103809101038734F0F01092010390915A0189E1989FC00111246AE070E00E942C
S12347E0CD3E6B5F87B5861730F4E7E4F0E080818F5F808308C087B5681728F4E7E4F0E01C
S12348008081815080837894FF91EF91BF91AF919F918F917F916F915F910F900FBE0F90B8
S12348201F9018951F920F920FB60F9211248F939F93AF93BF93EF93FF93F8948091E202AE
S12348409091E302A091E402B091E5020097A105B10541F0EBE2F0E080818F7D808380813D
S12348608F7E80837894FF91EF91BF91AF919F918F910F900FBE0F901F901895E1EBF0E025
S12348801082A0E7B0E08C9181608C9380818760808381E08093B20008951F920F920FB689
S12348A00F9211248F939F93AF93BF9381E0809324028091A9019091AA01A091AB01B091F7
S12348C0AC014296A11DB11D8093A9019093AA01A093AB01B093AC01809102038F5F809352
S12348E00203BF91AF919F918F910F900FBE0F901F9018951F920F920FB60F9211248F9359
S12349009F93EF93FF9380910003813051F410920003E8E8F0E0808191818C599F4F918304
S12349208083FF91EF919F918F910F900FBE0F901F9018951F920F920FB60F9211240F901D
S12349400FBE0F901F9018951F920F920FB60F9211240F900FBE0F901F9018951F920F92E5
S12349600FB60F9211240F900FBE0F901F9018951F920F920FB60F9211242F933F935F93BE
S12349806F937F938F939F93AF93BF93EF93FF93E4E8F0E020813181118210828091CF010E
S12349A09091D001880F991F880F991F820F931F880F991F6AE070E00E94CD3E862F972F0F
S12349C09093D0018093CF01FF91EF91BF91AF919F918F917F916F915F913F912F910F90DD
S12349E00FBE0F901F9018951092800088E893E1909389008093880080E197E290938B0016
S1234A0080938A00E1E8F0E080E8808383E08083EFE6F0E0808181608083E9E6F0E0808161
S1234A208A608083EDE3F0E0808183608083089588E98093C1008FE08093C4008AEA95E0ED
S1234A409093760580937505909372058093710588E795E090937405809373059093DD05F4
S1234A608093DC05109277051092240508951F920F920FB60F9211248F939F93EF93FF9363
S1234A8080917705882311F1E0917505F091760581918093C600F0937605E0937505EC5DD2
S1234AA0F54030F08AEA95E090937605809375058091770581508093770580917705882364
S1234AC029F4E1ECF0E080818F7D8083FF91EF919F918F910F900FBE0F901F9018951F9290
S1234AE00F920FB60F9211242F938F939F93EF93FF938091C600E091DC05F091DD058083BD
S1234B00809124058F5F809324058091DC059091DD0501969093DD058093DC058A5A9540EF
S1234B2030F088E795E09093DD058093DC05FF91EF919F918F912F910F900FBE0F901F909A
S1234B40189580912405882319F42FEF3FEF1AC0F89480912405815080932405E0917305D0
S1234B60F09174052191F0937405E0937305EA5AF54030F088E795E09093740580937305FA
S1234B80789430E0822F932F0895982F80917705823310F080E00895F894809177058F5FD8
S1234BA080937705E0917105F0917205908380917105909172050196909372058093710597
S1234BC08C5D954030F08AEA95E09093720580937105E1ECF0E0808180628083789481E0F7
S1234BE00895CF93DF93EC0104C00E94C5258111219688818823C9F781E0DF91CF91089578
S1234C0089ED91E00E94F12508958091240508958F929F92AF92BF92CF92DF92EF92FF92B5
S1234C200F931F93DF93CF93CDB7DEB729970FB6F894DEBF0FBECDBF8C01F62EE42EDE0186
S1234C401196ECEDF1E089E001900D928150E1F749E00F2EF9E0AF2EBB24F02D6E0108949A
S1234C60C11CD11C0F2EFEE28F2EF02D9924FF2071F09501241B31098F2D90E02817390778
S1234C8030F04150F601E40FF11D8082F92C4150F601E40FF11DC8016AE070E00E94CD3EA7
S1234CA0805D8083C8016AE070E00E94CD3E862F972F8C010115110511F4FF2019F085E03A
S1234CC08F15A8F689E0182F1E19193068F47E010894E11CF11CF701E10FF11D80810E9444
S1234CE0C5251F5F1930B8F329960FB6F894DEBF0FBECDBFCF91DF911F910F91FF90EF9020
S1234D00DF90CF90BF90AF909F908F900895EF92FF920F931F93FC018C010F5F1F4F80817B
S1234D200E94C52578010894E11CF11CF80180810E94C525F70180810E94C525F7018181BF
S1234D400E94C5251F910F91FF90EF900895282F392FEFE3F0E0808181FDFDCF822F932FA9
S1234D6092BD81BDF89A80B50895262F372FA901BA016F5F7F4FDC019D91EFE3F0E08081D4
S1234D8081FDFDCF1FBA52BD41BD90BD0FB6F894FA9AF99A0FBEAB014F5F5F4F2D91EFE3B5
S1234DA0F0E0808181FDFDCF1FBA72BD61BD20BD0FB6F894FA9AF99A0FBE2C91EFE3F0E02D
S1234DC0808181FDFDCF1FBA52BD41BD20BD0FB6F894FA9AF99A0FBE11962C91EFE3F0E076
S1234DE0808181FDFDCF1FBACA01019692BD81BD20BD0FB6F894FA9AF99A0FBE08952F921C
S1234E003F924F925F926F927F928F929F92AF92BF92CF92DF92EF92FF920F931F93DF934B
S1234E20CF93CDB7DEB762970FB6F894DEBF0FBECDBF9A8B898BDC011C966D917D918D91C1
S1234E409C911F97FD01E059FF4F20813181428153810E940F3C20E030E040E050E00E940D
S1234E60743C882309F450C0E989FA89E85BFF4FFA87E987A080B180C280D380AD82BE82FA
S1234E80CF82D886E989FA896485758586859785E059FF4F2081318142815381A989BA897A
S1234EA09496ED90FD900D911C9197971896AD90BD90CD90DC901B97D8962D903D904D90B9
S1234EC05C90DB970E940F3C3B014C01C801B701A60195010E940C3EA20191010E940F3C2E
S1234EE09B01AC01C401B3010E940C3E9B01AC016D817E818F8198850E940F3CE985FA85C3
S1234F006083718382839383A989BA891C96AD90BD90CD90DC901F9794966D917D918D9117
S1234F209C91979718962D913D914D915C911B97D896ED90FD900D911C91DB970E940C3E3A
S1234F40A80197010E940F3C9B01AC01C601B5010E940C3EE989FA89EC5BFF4FFC87EB87EE
S1234F606083718382839383E989FA89E459FF4F6081718182819381E989FA89E45BFF4F4F
S1234F80FE87ED872081318142815381E989FA89E859FF4F2080318042805380A989BA894B
S1234FA0D896AD90BD90CD90DC90DB97FD01E45AFF4FE080F180028113810E940C3E3B0120
S1234FC04C01C601B501A80197010E940F3C9B01AC01C201B1010E940C3E9B01AC01C4011D
S1234FE0B3010E940F3CED85FE856083718382839383AB85BC856D917D918D919C91E989EB
S1235000FA89E85BFF4F2081318142815381ED85FE85E080F180028113810E94103CA8011A
S123502097010E94103CE989FA89E85AFF4F6083718382839383A989BA898C91882309F435
S12350405FC0A85BBF4FB88BAF872D903D904D905C90E989FA89E05AFF4FE080F18002817F
S12350601381E989FA89608571858285938520AD31AD42AD53ADEC59FF4FA080B180C280E9
S1235080D380A982BA82CB82DC82E989FA89EC5AFF4F6080718082809380E989FA89E85A01
S12350A0FF4FA080B180C280D3800E940F3C9B01AC01C801B7010E940C3E9B01AC01C20109
S12350C0B1010E94103C7B018C01C401B301A60195010E940F3C9B01AC0169817A818B8146
S12350E09C810E940C3E9B01AC01C801B7010E94103CAF85B8896D937D938D939C9313976D
S1235100E989FA898481813009F07DC0E85AFF4F2081318142815381A989BA899896ED9010
S1235120FD900D911C919B9760E070E088EC92E40E940F3CA80197010E94743C88236CF45C
S1235140E989FA8980A591A5A2A5B3A5EC5AFF4F80839183A283B3833FC0E989FA89E85A20
S1235160FF4F2081318142815381A989BA899C96ED90FD900D911C919F9760E070E088ECBD
S123518092E40E940F3CA80197010E94C33D18166CF4E989FA8984A595A5A6A5B7A5EC5AF2
S12351A0FF4F80839183A283B38316C0E989FA89E85AFF4F208131814281538160E070E056
S12351C088EC92E40E940F3CE989FA89EC5AFF4F6083718382839383E989FA89EC5AFF4FF0
S12351E0608171818281938126E636ED43E254E40E940C3E0E94E53CE989FA89E458FF4F07
S12352007183608368C0E989FA89E85AFF4F6081718182819381A989BA8998962D913D91ED
S12352204D915C919B970E94743C88236CF4E989FA8980A591A5A2A5B3A5EC5AFF4F80838A
S12352409183A283B38331C0E989FA89E85AFF4F6081718182819381A989BA899C962D9116
S12352603D914D915C919F970E94C33D18166CF4E989FA8984A595A5A6A5B7A5EC5AFF4F98
S123528080839183A283B38310C0E989FA89E85AFF4F80819181A281B381E989FA89EC5A9E
S12352A0FF4F80839183A283B383E989FA89EC5AFF4F608171818281938120E030E04BE17B
S12352C054E40E940C3E0E94E53CE989FA89E458FF4F71836083E989FA8980AD91ADA2ADDE
S12352E0B3ADE45AFF4F80839183A283B383E989FA8984859585A685B785E059FF4F808343
S12353009183A283B383A989BA8911968C9162960FB6F894DEBF0FBECDBFCF91DF911F9122
S12353200F91FF90EF90DF90CF90BF90AF909F908F907F906F905F904F903F902F9008950A
S1235340EF92FF920F931F93CF93DF93EC01FC01E258FF4F0190F081E02D9881AFE3B0E053
S12353608C9181FDFDCF1FBAF2BDE1BD90BD0FB6F894FA9AF99A0FBEFE01E258FF4F0190F2
S1235380F081E02D2981AFE3B0E08C9181FDFDCF1FBACF01019692BD81BD20BD0FB6F8945D
S12353A0FA9AF99A0FBEFE01E258FF4F0190F081E02D2C81AFE3B0E08C9181FDFDCF1FBA50
S12353C0CF01049692BD81BD20BD0FB6F894FA9AF99A0FBEFE01E258FF4F0190F081E02D1A
S12353E02D81AFE3B0E08C9181FDFDCF1FBACF0105960F2EF1E4EF2EFF24F02DF7019183B3
S1235400808320BD0FB6F894FA9AF99A0FBE8E0102581F4FF80160817181685F7F4FCE01DC
S1235420C0960E94B526F80160817181645F7F4FCE0108960E94B526F80160817181605FC3
S12354407F4FCE010C960E94B526F801608171816C5E7F4FCE0140960E94B526F80160812C
S12354607181685E7F4FCE0144960E94B526F80160817181645E7F4FCE0148960E94B526F6
S1235480F80160817181605E7F4FCE018C589F4F0E94B526F801608171816C5D7F4FCE0160
S12354A080960E94B526F80160817181685D7F4FCE0184960E94B526F80160817181645D03
S12354C07F4FCE0188960E94B526F80160817181605D7F4FCE018C960E94B526F8016081F1
S12354E071816C5C7F4FCE01C4960E94B526F80160817181685C7F4FCE01805C9F4F0E94E1
S1235500B52612BCF7011082DF91CF911F910F91FF90EF900895CF92DF92EF92FF920F9303
S12355201F938C0182E80E94C52588E50E94C525F8018081880F0E94C525F80181810E947F
S1235540C525F80182810E94C525F80183810E94C525F80184810E94C525F80185810E9421
S1235560C525F80186810E94C52580E00E94C5250F2EFFEFCF2EFFE8DF2EF0E0EF2EF0E0EC
S1235580FF2EF02DD701C6010197A109B109000001F0D1F7C8950000C801C0960E9487269E
S12355A0C80108960E948726C8010C960E948726D701C6010197A109B109000001F0D1F723
S12355C0C8950000C80140960E948726C80144960E948726C80148960E948726D701C601F5
S12355E00197A109B109000001F0D1F7C8950000C8018C589F4F0E948726C80180960E942A
S12356008726C80184960E948726D701C6010197A109B109000001F0D1F7C8950000C8012D
S123562088960E948726C8018C960E948726C801C4960E948726D701C6010197A109B109B2
S1235640000001F0D1F7C8950000C801CC960E948726C801C8960E948726C801805C9F4FAD
S12356600E948726D701C6010197A109B109000001F0D1F7C8950000C8018C5B9F4F0E94E6
S12356808726C801885B9F4F0E948726C801845B9F4F0E948726D701C6010197A109B109F0
S12356A0000001F0D1F7C8950000C8018C599F4F0E948726C8018C5A9F4F0E9487268DE785
S12356C00E94C5251F910F91FF90EF90DF90CF900895DF93CF9300D000D0CDB7DEB7BC0127
S12356E0CE01019644E050E027EA36E20E94AC3B29813A814B815C81622F732F842F952F82
S12357000F900F900F900F90CF91DF9108952F923F924F925F926F927F928F929F92AF9293
S1235720BF92CF92DF92EF92FF920F931F93DF93CF9300D000D0CDB7DEB79C838B8381E0C1
S1235740AB81BC818C9314961C9280E090E0A0E4BFE3EB81FC8184879587A687B7878DEC7B
S12357609CECACECBEE3EB81FC81808B918BA28BB38B20E030E040E050E0AB81BC81549636
S12357802D933D934D935C935797EB81FC81208F318F428F538F80E090E0A0E8BFE3EB8147
S12357A0FC81848F958FA68FB78F80E090E0A0E8B0E4EB81FC8180A391A3A2A3B3A383E389
S12357C093E3A3E3BFE3EB81FC8184A395A3A6A3B7A380E090E0A0EFB1E4EB81FC8180A738
S12357E091A7A2A7B3A780E090E0ACE8B2E4EB81FC8184A795A7A6A7B7A780E090E0A0E283
S1235800B2E4EB81FC8180AB91ABA2ABB3AB80E090E0A0EAB0E4EB81FC8184AB95ABA6AB5C
S1235820B7ABAB81BC81D8962D933D934D935C93DB97EB81FC8124AF35AF46AF57AFEB8153
S1235840FC81E05CFF4F80E090E0A0E8BEE380839183A283B383EB81FC8180899189A2899B
S1235860B389EC58FF4F80839183A283B383EB81FC81E85BFF4F2083318342835383EB810C
S1235880FC81E45AFF4F2083318342835383EB81FC81E258FF4F0190F081E02DAFE3B0E067
S12358A08C9181FDFDCFCF01049692BD81BDF89A80B5AB81BC8114968C93149714968C911B
S12358C01497853030F014961C928B819C810E94A029EB81FC81E258FF4F0190F081E02DD8
S12358E0AFE3B0E08C9181FDFDCFF2BDE1BDF89A80B5EB81FC818083EB81FC81E258FF4FAA
S12359000190F081E02DAFE3B0E08C9181FDFDCFCF01019692BD81BDF89A80B5AB81BC81C7
S123592011968C931197FD01E258FF4F0190F081E02DAFE3B0E08C9181FDFDCFCF0102966F
S123594092BD81BDF89A80B5EB81FC818283EB81FC81E258FF4F0190F081E02DAFE3B0E05F
S12359608C9181FDFDCFCF01039692BD81BDF89A80B5AB81BC8113968C931397FD01E258EC
S1235980FF4F0190F081E02DAFE3B0E08C9181FDFDCFCF01049692BD81BDF89A80B5EB81F3
S12359A0FC818483EB81FC81E258FF4F0190F081E02DAFE3B0E08C9181FDFDCFCF010596EB
S12359C092BD81BDF89A80B5AB81BC8115968C93159781E08C9314968C911497882321F0E2
S12359E081E014968C9303C0EB81FC811482AB81BC8114961C921497FD01E258FF4F0190B4
S1235A00F081E02DAFE3B0E08C9181FDFDCFCF0106960F2EF1E4EF2EFF24F02DF701918394
S1235A208083F89A80B5AB81BC8116968C9316978D0102581F4FF8018081918108960E9415
S1235A40692BAB81BC81D0966D937D938D939C93D397F801808191810C960E94692BAB8106
S1235A60BC8118966D937D938D939C931B97F8018081918140960E94692BAB81BC811C96F3
S1235A806D937D938D939C931F97EB81FC8184859585A685B785E059FF4F80839183A283B7
S1235AA0B383D8018D919C9144960E94692BEB81FC81608B718B828B938BD8018D919C9159
S1235AC048960E94692BEB81FC81648B758B868B978BD8018D919C914C960E94692BEB81FB
S1235AE0FC81608F718F828F938FD8018D919C9180960E94692BEB81FC81EC58FF4F608335
S1235B00718382839383F8018081918184960E94692BAB81BC8190966D937D938D939C9328
S1235B209397F8018081918188960E94692BAB81BC8194966D937D938D939C939797F801BE
S1235B40808191818C960E94692BAB81BC8198966D937D938D939C939B97F80180819181A2
S1235B60C0960E94692BAB81BC819C966D937D938D939C939F97F80180819181C4960E945D
S1235B80692BAB81BC81D4966D937D938D939C93D797F80180819181C8960E94692BEB81C1
S1235BA0FC81E05CFF4F608371838283938312BCD7011C9260817181828193812FE632E182
S1235BC043E85AE30E94743C882364F4EB81FC81E05CFF4F8FE692E1A3E8BAE3808391836A
S1235BE0A283B383EB81FC81608971898289938920E030E040E050E00E94743C181654F02F
S1235C0080E090E0A0E2B1E4EB81FC81808B918BA28BB38BEB81FC81EC58FF4F60817181D0
S1235C208281938120E030E040E050E00E94743C181664F0EB81FC81EC58FF4F80E090E0CA
S1235C40A0E2B1E480839183A283B383EB81FC81E05CFF4F608171818281938120E030E04A
S1235C6040E050E00E94743C181664F0EB81FC81E05CFF4F80E090E0A0E8BFE38083918378
S1235C80A283B383AB81BC8190966D917D918D919C91939720E030E040E050E00E94743CE3
S1235CA0181654F080E090E0A0E2B1E4EB81FC8180A391A3A2A3B3A3AB81BC81D4966D91DB
S1235CC07D918D919C91D79720E030E040E050E00E94743C181654F080E090E0A0E2B1E4EE
S1235CE0EB81FC8184AB95ABA6ABB7ABAB81BC811C966D917D918D919C911F97A05CBF4F63
S1235D00BA83A9832D913D914D915C91EB81FC81E088F188028913890E940C3EA8019701A1
S1235D200E94783CEB81FC81E05AFF4F6083718382839383A981BA816D917D918D919C91EA
S1235D40EB81FC81EC58FF4F20813181428153810E94783CEB81FC81EC59FF4F6083718331
S1235D6082839383EB81FC81648575858685978520A131A142A153A1E488F588068917898F
S1235D802488358846885788A0A0B1A0C2A0D3A0A981BA816D907D908D909C900E940C3EDF
S1235DA0A80197010E940C3E7B018C01C601B501A40193010E940C3E9B01AC01C201B10149
S1235DC00E94103C9B01AC01C801B7010E94783CEB81FC81E859FF4F608371838283938347
S1235DE0EB81FC81A488B588C688D788E488F5880689178960A171A182A193A1A981BA81B9
S1235E002D913D914D915C910E940C3E9B01AC01C801B7010E94103C9B01AC01C601B501BD
S1235E200E94783CEB81FC81E459FF4F60837183828393830F900F900F900F90CF91DF9156
S1235E401F910F91FF90EF90DF90CF90BF90AF909F908F907F906F905F904F903F902F90CC
S1235E600895282F392FEFE3F0E0808181FDFDCF822F932F92BD81BDF89A80B50895AF9230
S1235E80BF92CF92DF92EF92FF920F931F93CF93DF938091A2029091A302A091A402B0910E
S1235EA0A502A8958091DE05853809F494C08638C0F48B3579F18C3550F4843309F442C49D
S1235EC0853509F4EAC0833309F048C438C4813809F471C0833809F4D8C2803809F03EC4BA
S1235EE0B8C2833909F447C4843950F48A3809F4F9C0813909F49CC1883809F02FC416C150
S1235F00883909F4D5C1893909F421C4853909F025C468C28CE50E94C52584E10E94C525CD
S1235F20C0E0D0E00F2EF3E1EF2EF4E0FF2EF02D0F2EFCECCF2EFCE1DF2EF02DCE01880F32
S1235F40991F880F991F8701080F191FF80180819181A281B3810E94C525F8018081918164
S1235F60A281B381892F9A2FAB2FBB270E94C525F80180819181A281B381CD01AA27BB2719
S1235F800E94C525F80180819181A281B3818B2F9927AA27BB270E94C525C6010197F1F70E
S1235FA0000000002196C530D10509F0C7CF83EA0E94C525E0C382E08093DE0580912202A3
S1235FC090E09695982F8827979587958D5E9C4F0E948B2AD0C3A0EEB5E0FD013191208120
S1235FE0922F80E07C01E30EF11C11978C91823009F43BC020E030E00F2EFEEDCF2EF5E088
S1236000DF2EF02DAFE3B0E001E410E060E470E04CEC5CE10F2EFFEDAF2EF5E0BF2EF02D6D
S1236020A895F601E20FF31F3496E0818C9181FDFDCF1C92C9018E0D9F1DE80199838883B4
S1236040EB01E8830FB6F894FA9AF99A0FBECA010197F1F7000000002F5F3F4FF501808142
S123606090E0029728173907D8F286E80E94C52584E00E94C52581E00E94C5258E2D0E9496
S1236080C5258F2D0E94C5258091DF0582500E94C52589E70E94C5256EC3E0EEF5E0919185
S12360A08081182F00E0090F111DC80161E37FE20E94C83BF82EE92E85E50E94C52584E0C4
S12360C00E94C5258F2D0E94C5258E2D0E94C525802F0E94C525812F0E94C5258AEA0E9414
S12360E0C52549C3E0EEF5E031912081922F80E0EC01C30FD11D8BE80E94C52583E00E94CE
S1236100C525EFE3F0E0808181FDFDCFD2BDC1BDF89A80B50E94C5258C2F0E94C5258D2F41
S12361200E94C52584E70E94C52525C389E80E94C52580E10E94C5250F2EFFE3EF2EF2E0F8
S1236140FF2EF02DE701888199810E94C52588819981892F0E94C525870104501040F801CE
S1236160808191810E94C525E80188819981892F0E94C52587010C5F1F4FF80180819181BF
S12361800E94C525E80188819981892F0E94C52587010E501040F801808191810E94C52551
S12361A0E80188819981892F0E94C52582E39BE20197F1F70000C89587010C501040F8019F
S12361C0808191810E94C525E80188819981892F0E94C52587010A501040F801808191818E
S12361E00E94C525E80188819981892F0E94C525870108501040F801808191810E94C525F7
S1236200E80188819981892F0E94C525EAEFFFEFEE0EFF1EE701888199810E94C5258881AA
S12362209981892F0E94C52586E70E94C525A3C282E90E94C52580E10E94C5258091220285
S123624090E09695982F88279795879503E113E089599C4F0E9487268091220290E096951E
S1236260982F882797958795C896800F911F0E9487268091220290E09695982F88279795FE
S123628087950896800F911F0E9487268091220290E09695982F882797958795885B9F4F53
S12362A0800F911F0E9487268DE60E94C52563C287E90E94C52581E10E94C5250F2EF3E32B
S12362C0EF2EF2E0FF2EF02DF701808191810E94C5258701E70189919991892F0E94C525F2
S12362E0888199810E94C52588819981892F0E94C5250C5F1F4FF801808191810E94C52513
S1236300E80188819981892F0E94C5258091A2029091A302A091A402B091A5020E94C52563
S123632060914B0370914C0380914D0390914E0320E030E040E251E40E940C3E0E94E53CE1
S1236340DC01CB010E94C5258701025F1F4FF801808191810E94C525E80188819981892F51
S12363600E94C52587B52AE0829FC0011124C29769E170E00E94E13E862F0E94C52586E6CF
S12363809EE00197F1F70000F7017096808191816AE070E00E94CD3E862F0E94C525ECE096
S12363A0F0E0EE0EFF1EE701888199810E94C52588819981892F0E94C52580911E0590919D
S12363C01F050E94C52580911E0590911F05892F0E94C52580918F020E94C52588E60E940E
S12363E0C525C9C186E90E94C52580E10E94C5258091220290E09695982F882797958795AF
S123640003E113E089599C4F0E94872685E892E00E9487268091220290E09695982F882711
S1236420979587950896800F911F0E9487268091220290E09695982F882797958795885B73
S12364409F4F800F911F0E94872689E60E94C52592C18091E0058093220280912202882361
S123646031F080912202813011F01092220280E80E94C52581E00E94C525809122020E9492
S1236480C5258FE70E94C52576C184E80E94C52584E20E94C52580910D0190910E010E94FA
S12364A0C52580910D0190910E01892F0E94C52580910F010E94C525809110010E94C52500
S12364C00FEF17E4C8010197F1F7000000C080911101909112010E94C5258091110190918F
S12364E01201892F0E94C52580913301909134016AE070E00E94CD3E862F0E94C52580910D
S12365003301909134016AE070E00E94CD3E872F0E94C52580911301909114016AE070E06F
S12365200E94CD3E862F0E94C52580911301909114016AE070E00E94CD3E872F0E94C52585
S123654080911501909116016AE070E00E94CD3E862F0E94C525C8010197F1F7000000C047
S123656080911501909116016AE070E00E94CD3E872F0E94C52580911701909118016AE082
S123658070E00E94CD3E862F0E94C52580911701909118016AE070E00E94CD3E872F0E94B7
S12365A0C52580911B0190911C016AE070E00E94CD3E862F0E94C52580911B0190911C018F
S12365C06AE070E00E94CD3E872F0E94C52580915701909158010E94C52580915701909135
S12365E05801892F0E94C525C8010197F1F7000000C080911D0190911E016AE070E00E9446
S1236600CD3E862F0E94C52580911D0190911E016AE070E00E94CD3E872F0E94C525809121
S12366203501909136016AE070E00E94CD3E862F0E94C52580913501909136016AE070E007
S12366400E94CD3E872F0E94C52580911F01909120010E94C52580911F0190912001892F1D
S12366600E94C525C8010197F1F7000000C0809123010E94C525809124010E94C5258091ED
S12366802501909126016AE070E00E94CD3E862F0E94C52580912701909128016AE070E0E3
S12366A00E94CD3E862F0E94C52580912B010E94C52580912C010E94C525C8010197F1F70C
S12366C0000000C080912D0190912E016AE070E00E94CD3E862F0E94C52580912D0190917F
S12366E02E016AE070E00E94CD3E872F0E94C52580912F01909130016AE070E00E94CD3E04
S1236700862F0E94C52580912F01909130016AE070E00E94CD3E872F0E94C52580913101D5
S1236720909132010E94C5258091310190913201892F0E94C5258BE70E94C5251CC00E941E
S1236740830219C00E9482070E945D0A14C0F894E091ED01F091EE0109950DC08EE80E94F1
S1236760C52581E00E94C5258091DE050E94C52581E70E94C525EEEDF5E0119280818823CB
S123678091F020E030E04EED55E0DA011196FA01E20FF31F329610822F5F3F4F8C9190E071
S12367A028173907A0F31092DF05DF91CF911F910F91FF90EF90DF90CF90BF90AF90089516
S12367C0AF92BF92CF92DF92EF92FF920F931F93CF93DF93382F492FC62E2DE088E190E05E
S12367E00FB6F894A895809360000FBE20936000662309F4C0C0D32E232F342FE9010F2ED1
S1236800FFEDEF2EF5E0FF2EF02D0EED15E0AA246894A1F8BB24B39480910303882309F018
S12368205FC08881F80180838081833309F447C08081843309F443C08081853509F43FC006
S123684080818835E1F180818B35C9F180818136B1F18081853699F180818F3681F1808150
S1236860803769F18081873751F18081893739F18081803821F180818A3709F180818138D6
S1236880F1F080818338D9F080818438C1F080818538A9F08081883891F080818A3879F05B
S12368A08081813961F08081833949F08081853931F08081883919F08081893919F4B09215
S12368C0030353C08FE80E94C5258B2D0E94C525F80180810E94C52580E70E94C52545C0D6
S12368E080910303813059F48881F70180838081833310F010920303A092030336C020913D
S12369000303F701808130E090E002962817390791F4F80180818095809303039091030309
S12369208881891729F4109203030E943F2F1DC0109203031AC0809103038230B0F020915C
S12369400303F701808130E090E002962817390764F4809103039881F801E80FF11D908304
S1236960809103038F5F8093030321969E012D192C1508F451CFDF91CF911F910F91FF904D
S1236980EF90DF90CF90BF90AF90089500000000000000000000000000000000000000007B
S12369A000000000000000000000000090E02091160630911706280F391F22953295307FFC
S12369C03227207F3227282B392B2F703F70E8E2F0E080818061808380818F7B808348E0A8
S12369E0AFE5B0E080818F7E808380818F7D80839C9191709295990F907E80818F7D892B82
S1236A0080830000000000000000000000000000000000000000000000000000000000006F
S1236A200000808180618083415000000000000000000000000000000000000000000000DC
S1236A4000000000000000000000442389F000000000000000000000000000000000000052
S1236A600000000000000000000000000000BACF40E1E8E2F0E0AFE5B0E080818F7E808399
S1236A8080818F7D8083369527959C9191709295990F907E80818F7D892B808380818061AA
S1236AA080834150000000000000000000000000000000000000000000000000000000003E
S1236AC00000000000000000000000000000000000000000000000000000000000000000B2
S1236AE0000000000000000000000000000000000000000000000000000000000000000092
S1236B0000000000442309F0B8CF3093170620931606E8E2F0E08081806480838081806177
S1236B2080836A3F39F480E791E00197F1F70000000008958CEC9CE10197F1F7000000000E
S1236B40089580910703E4E1F2E0E80FF11D808190910603890F68EF0E94C6340895809377
S1236B600603609307030E94A135089510920603809107038F5F80930703823010F01092D1
S1236B8007030E94A13508958A3029F40E94B6350E94A13508956AEF0E94C634809106034A
S1236BA08F5F809306030895CF93DF93FC01009751F08081882339F0EF010E94C43521966A
S1236BC088818823D1F7DF91CF9108956AEF0E94C634089588E368EF0E94C63408958BE3CD
S1236BE068EF0E94C634089581E068EF0E94C634109206031092070308950F931F93E7E29C
S1236C00F0E080818064808380818061808380818062808310921306E8E2F0E080818064B3
S1236C2080838081806180838FEF97EDA0E0B0E00197A109B109000001F0D1F7C895000044
S1236C4081E068EF0E94C6340CEC1CE1C8010197F1F70000000088E368EF0E94C6348FE0D1
S1236C6068EF0E94C63486E068EF0E94C63481E068EF0E94C634C8010197F1F70000000027
S1236C801F910F9108950E94FD350E94B6358FEE91E00E94D43508958F929F92AF92BF9288
S1236CA0CF92DF92EF92FF920F931F93DF93CF93CDB7DEB729970FB6F894DEBF0FBECDBFA4
S1236CC08C01F62EE42EDE011196EBE0F2E089E001900D928150E1F749E00F2EF9E0AF2E6C
S1236CE0BB24F02D6E010894C11CD11C0F2EFEE28F2EF02D9924FF2071F09501241B31097C
S1236D008F2D90E02817390730F04150F601E40FF11D8082F92C4150F601E40FF11DC801A2
S1236D206AE070E00E94CD3E805D8083C8016AE070E00E94CD3E862F972F8C0101151105E4
S1236D4011F4FF2019F085E08F15A8F689E0182F1E19193068F47E010894E11CF11CF701B2
S1236D60E10FF11D80810E94C4351F5F1930B8F329960FB6F894DEBF0FBECDBFCF91DF912D
S1236D801F910F91FF90EF90DF90CF90BF90AF909F908F9008958F929F92AF92BF92CF9205
S1236DA0DF92EF92FF920F931F93DF93CF93CDB7DEB72A970FB6F894DEBF0FBECDBF8C0176
S1236DC0F62E842EDE011196E2E0F2E089E001900D928150E1F7112314F01A8607C0109539
S1236DE001951F4F8DE2898381E08A8749E00F2EF9E0AF2EBB24F02D6E010894C11CD11CB1
S1236E000F2EFEE29F2EF02DEE24FF2071F09501241B31098F2D90E02817390730F041506A
S1236E20F601E40FF11D9082FE2C4150F601E40FF11DC8016AE070E00E94E13E805D80838D
S1236E40C8016AE070E00E94E13E862F972F8C010115110511F4FF2019F085E08F15A8F602
S1236E608A858130A1F498E0BE016F5F7F4F292F30E0FB01E20FF31F8081803231F4FE01A8
S1236E80E20FF31F8DE2818302C09150F0CF89E0182F1819193068F47E010894E11CF11C6B
S1236EA0F701E10FF11D80810E94C4351F5F1930B8F32A960FB6F894DEBF0FBECDBFCF9163
S1236EC0DF911F910F91FF90EF90DF90CF90BF90AF909F908F900895EFE3F0E0808181FD78
S1236EE0FDCF84E893E092BD81BDF89A80B580931203EFE3F0E0808181FDFDCF85E893E09A
S1236F0092BD81BDF89A80B580932505EFE3F0E0808181FDFDCF86E893E092BD81BDF89AEF
S1236F2080B580933E05EFE3F0E0808181FDFDCF87E893E092BD81BDF89A80B580932D045B
S1236F40089580911203882359F480912505813039F480913E0590E0823019F491E001C0A4
S1236F6090E0892F089580912D04811181E00895AF92BF92CF92DF92EF92FF920F931F93AC
S1236F80CF93DF93982F7A018B01E90180910803891721F010921C0690930803943109F4E0
S1236FA047C0953140F4992381F0892F8950823008F0DDC017C0903209F47CC0983209F42E
S1236FC095C09E3109F0D3C054C082E390E09B8B8A8B81E090E09987888784EF91E09D8BCD
S1236FE08C8BC5C0CC24DD246894C3F8CC0EDD1EC801B7012CEB32E040E050E00E94F43EA6
S1237000F60131832083215233402CF080E293E0F6019183808380911C0624E333E0281BA9
S123702031093D8B2C8B82E390E09B8B8A8B9FC0FE0138968EE591E09183808380911C0629
S123704090E0880F991F82549F4F9183808320911C0684E393E0821B91099D8B8C8B80915E
S12370601C066FE00E94C13E90E0C2969B8B8A8B7EC0FE0138968EE591E0918380838091E0
S12370801C0690E0880F991F82549F4F9183808320911C0684E393E0821B91099D8B8C8B0D
S12370A080911C0664E10E94C13E90E0CC969B8B8A8B5DC0FE0138968EE591E091838083C1
S12370C080911C0690E0880F991F82549F4F9183808320911C0684E393E0821B91099D8BD3
S12370E08C8B82E390E09B8B8A8B41C0FE01389682E593E09183808380911C0690E0880F6C
S1237100991F909581959F4F8E5A9C4F9183808380911C0690E088539F4F9D8B8C8B0F2EB8
S1237120F2E1AF2EBB24F02DAC0EBD1EF501C080D180F3E3CF16D104D4F0C801B70124EF9B
S123714031E040E050E00E94F43E8091180690911906A0911A06B0911B06281739074A0704
S12371605B0769F1C6010197F50191838083C801B70124EF31E040E050E00E94F43E822F69
S1237180932FA42FB52F9C01AD018091180690911906A0911A06B0911B06281739074A0735
S12371A05B0769F080911C068F5F80931C06209318063093190640931A0650931B068A89FD
S12371C09B899C01220F331F880F991F880F991F880F991F280F391F3F8B2E8BDF91CF9198
S12371E01F910F91FF90EF90DF90CF90BF90AF900895282F392FEFE3F0E0808181FDFDCF88
S1237200822F932F92BD81BDF89A80B50895282F392FEFE3F0E0808181FDFDCF1FBA822FD0
S1237220932F92BD81BD60BD0FB6F894FA9AF99A0FBE0895CF92DF92EF92FF920F931F93C4
S1237240CF93DF93C0E0D0E004EA16E00F2EFEE2CF2EF4E0DF2EF02D0F2EF7E0EF2EF9E3FD
S1237260FF2EF02DA895CE01880F991FF601E80FF91F60817181C801A7010E94FA3B21968D
S12372800E5F1F4FC837D10569F76091200570912105809122059091230520E030E040E2EA
S12372A051E40E940C3E0E94E53C9B01AC0180EA96E0B90147E059E30E94FA3BDF91CF91F9
S12372C01F910F91FF90EF90DF90CF900895EF92FF920F931F93CF93DF93EB018D3C91055C
S12372E040F4EEE2F4E08081918101969183808314C0885C904065E070E00E94CD3E683788
S123730008F067E7E62FF0E0EE0FFF1FE25DFB4F80819181019691838083609120057091C2
S12373202105809122059091230520E030E04EEB52E40E940C3E7B018C01BE01660F771F64
S1237340660F771F6C0F7D1F80E090E00E94113D9B01AC01C801B7010E94103C20E030E07F
S123736048EC52E40E94783C60932005709321058093220590932305809111038F5F80935D
S12373801103893720F00E941A3910921103DF91CF911F910F91FF90EF900895AF92BF92FD
S12373A0CF92DF92EF92FF920F931F93CF93DF93C0E0D0E004EA16E00F2EF9EFAF2EF8E3AC
S12373C0BF2EF02D0F2EFEE2CF2EF4E0DF2EF02DA895C801B5010E94C83B9E01220F331F04
S12373E0F601E20FF31F91838083808191818D5D9F4F40F0CE01880F991FF601E80FF91F39
S12374001182108221960E5F1F4FC837D10501F780EA96E069EF78E30E94C83B6AE070E012
S12374200E94CD3E80E090E00E94113D6093200570932105809322059093230560912005FF
S123744070912105809122059091230520E030E849E854E40E94C33D181664F480E090E8FF
S1237460AEE5B4E48093200590932105A0932205B0932305DF91CF911F910F91FF90EF9069
S1237480DF90CF90BF90AF900895EF92FF920F931F93CF93DF93C4E4D6E00F2EF3E1EF2E29
S12374A0F4E0FF2EF02D09EF18E3CE01845496408E0D9F1DBE0144E050E098010E94AC3BAE
S12374C0249686E0C835D80781F712BC11BCDF91CF911F910F91FF90EF900895EF92FF92BC
S12374E00F931F9303E114E00F2EF7E0EF2EF9E3FF2EF02D84E496E0B80144E050E0970182
S12375000E94DE3BB8016C5F7F4F88E496E044E050E097010E94DE3BB801685F7F4F8CE413
S123752096E044E050E097010E94DE3BB801645F7F4F80E596E044E050E097010E94DE3B5E
S1237540005F1F4F84E596E0B80144E050E097010E94DE3B1F910F91FF90EF900895EF929F
S1237560FF920F931F936091A9017091AA018091AB019091AC0120E63AEE40E050E00E9430
S1237580F43E790100E010E08091090390910A03A0910B03B0910C03E816F9060A071B0761
S12375A009F4C2C0E3E1F4E080819181A281B3812091090330910A0340910B0350910C03EC
S12375C0821B930BA40BB50B8E0D9F1DA01FB11F80839183A283B38380918F02853148F411
S12375E0833170F5893089F08A3051F1882369F077C0803251F0813220F48E3108F470C060
S12376003AC0883209F06CC051C0E7E1F4E080819181A281B3812091090330910A0340911A
S12376200B0350910C03821B930BA40BB50B8E0D9F1DA01FB11F80839183A283B38350C036
S1237640EBE1F4E080819181A281B3812091090330910A0340910B0350910C03821B930B87
S1237660A40BB50B8E0D9F1DA01FB11F80839183A283B38335C0EFE1F4E080819181A28170
S1237680B3812091090330910A0340910B0350910C03821B930BA40BB50B8E0D9F1DA01F98
S12376A0B11F80839183A283B3831AC0E3E2F4E080819181A281B3812091090330910A031C
S12376C040910B0350910C03821B930BA40BB50B8E0D9F1DA01FB11F80839183A283B383D5
S12376E080910D0390910E03A0910F03B09110034496A11DB11D8E159F05A007B10750F44C
S12377000E946E3AE0920D03F0920E0300930F031093100312BC11BCE0920903F0920A0303
S123772000930B0310930C031F910F91FF90EF9008950E946E3A1092090310920A031092AE
S12377400B0310920C0310920D0310920E0310920F03109210030895A0E0B0E0E2EBFBE340
S12377600C94203F7C01EB018A01690109C0CE012196F6010995F70181937F010150104097
S123778001151105A1F7CDB7DEB7E8E00C943C3FDF92EF92FF920F931F937B018C01FB0149
S12377A00995D82EC8010196F7010995982F8D2D1F910F91FF90EF90DF900895A0E0B0E030
S12377C0E4EEFBE30C94203FEC017B018A01690109C0CE012196F70161917F01F60109954A
S12377E00150104001151105A1F7CDB7DEB7E8E00C943C3FDF92EF92FF920F931F93D72E48
S12378007A018C01FA010995C80101966D2DF70109951F910F91FF90EF90DF900895505821
S1237820BB27AA270ED075C166D130F06BD120F031F49F3F11F41EF45BC10EF4E095E7FB4B
S123784051C1E92F77D180F3BA17620773078407950718F071F49EF58FC10EF4E0950B2E64
S1237860BA2FA02D0B01B90190010C01CA01A0011124FF27591B99F0593F50F4503E68F163
S12378801A16F040A22F232F342F4427585FF3CF469537952795A795F0405395C9F77EF431
S12378A01F16BA0B620B730B840BBAF09150A1F0FF0FBB1F661F771F881FC2F70EC0BA0F3A
S12378C0621F731F841F48F4879577956795B795F7959E3F08F0B3CF9395880F08F09927E8
S12378E0EE0F979587950895D9D008F481E008950CD00FC107D140F0FED030F021F45F3FAA
S123790019F0F0C0511139C1F3C014D198F39923C9F35523B1F3951B550BBB27AA2762175B
S12379207307840738F09F5F5F4F220F331F441FAA1FA9F333D00E2E3AF0E0E830D091500D
S12379405040E695001CCAF729D0FE2F27D0660F771F881FBB1F261737074807AB07B0E87E
S123796009F0BB0B802DBF01FF2793585F4F2AF09E3F510568F0B6C000C15F3FECF3983EE9
S1237980DCF3869577956795B795F7959F5FC9F7880F911D9695879597F90895E1E0660F6C
S12379A0771F881FBB1F621773078407BA0720F0621B730B840BBA0BEE1F88F7E095089570
S12379C004D06894B111D9C00895BCD088F09F5790F0B92F9927B751A0F0D1F0660F771F55
S12379E0881F991F1AF0BA95C9F712C0B13081F0C3D0B1E00895C0C0672F782F8827B85FA3
S1237A0039F0B93FCCF3869577956795B395D9F73EF490958095709561957F4F8F4F9F4F46
S1237A200895E89409C097FB3EF490958095709561957F4F8F4F9F4F9923A9F0F92F96E9D1
S1237A40BB279395F695879577956795B795F111F8CFFAF4BB0F11F460FF1BC06F5F7F4FC1
S1237A608F4F9F4F16C0882311F096E911C0772321F09EE8872F762F05C0662371F096E8AB
S1237A80862F70E060E02AF09A95660F771F881FDAF7880F9695879597F90895990F000816
S1237AA0550FAA0BE0E8FEEF16161706E807F907C0F012161306E407F50798F0621B730B61
S1237AC0840B950B39F40A2661F0232B242B252B21F408950A2609F4A140A6958FEF811DC1
S1237AE0811D089597F99F6780E870E060E008959FEF80EC089500240A941616170618065C
S1237B000906089500240A9412161306140605060895092E0394000C11F4882352F0BB0F5A
S1237B2040F4BF2B11F460FF04C06F5F7F4F8F4F9F4F089557FD9058440F551F59F05F3F0C
S1237B4071F04795880F97FB991F61F09F3F79F087950895121613061406551FF2CF469547
S1237B60F1DF08C0161617061806991FF1CF86957105610508940895E894BB2766277727D1
S1237B80CB0197F908958ADF08F48FEF08950EF0A6C0AECF6894A6CFD5DFC8F39923D1F327
S1237BA0C6F3DF93CF931F930F93FF92C92FDD2788232AF02197660F771F881FDAF720E053
S1237BC030E040E85FEB9FE3883920F0803E30F021968F7725DEE0E7F0E003C021DEEDE9FF
S1237BE0F0E08BD08B01BE01EC01FB2E6F5771097595771F880B990B16DF28E132E741E3A3
S1237C005FE316D0AF2D9801AE01FF900F911F91CF91DF9116DE7DCF0BD07BCF6CDF28F09D
S1237C2071DF18F0952309F05DCF62CF1124A5CF81DFA0F3959FD1F3950F50E0551F629FFD
S1237C40F001729FBB27F00DB11D639FAA27F00DB11DAA1F649F6627B00DA11D661F829F59
S1237C602227B00DA11D621F739FB00DA11D621F839FA00D611D221F749F3327A00D611D87
S1237C80231F849F600D211D822F762F6A2F11249F5750408AF0E1F088234AF0EE0FFF1FDB
S1237CA0BB1F661F771F881F91505040A9F79E3F510570F017CF61CF5F3FECF3983EDCF348
S1237CC0869577956795B795F795E7959F5FC1F7FE2B880F911D9695879597F908959F3FB3
S1237CE031F0915020F4879577956795B795880F911D9695879597F90895DF93CF931F93BB
S1237D000F93FF92EF92DF927B018C01689405C0DA2EEF018DDFFE01E894A59125913591DF
S1237D2045915591AEF3EF018CDDFE019701A801DA9479F7DF90EF90FF900F911F91CF913E
S1237D40DF910895629FD001739FF001829FE00DF11D649FE00DF11D929FF00D839FF00DD6
S1237D60749FF00D659FF00D9927729FB00DE11DF91F639FB00DE11DF91FBD01CF011124B2
S1237D800895991B79E004C0991F961708F0961B881F7A95C9F780950895AA1BBB1B51E16E
S1237DA007C0AA1FBB1FA617B70710F0A61BB70B881F991F5A95A9F780959095BC01CD01A4
S1237DC0089597FB092E07260AD077FD04D0E5DF06D000201AF4709561957F4F0895F6F7CF
S1237DE0909581959F4F0895A1E21A2EAA1BBB1BFD010DC0AA1FBB1FEE1FFF1FA217B30747
S1237E00E407F50720F0A21BB30BE40BF50B661F771F881F991F1A9469F760957095809566
S1237E2090959B01AC01BD01CF0108952F923F924F925F926F927F928F929F92AF92BF924B
S1237E40CF92DF92EF92FF920F931F93CF93DF93CDB7DEB7CA1BDB0B0FB6F894DEBF0FBE73
S1237E60CDBF09942A88398848885F846E847D848C849B84AA84B984C884DF80EE80FD808C
S1237E800C811B81AA81B981CE0FD11D0FB6F894DEBF0FBECDBFED010895F894FFCF2043F6
S1237EA0616C6962726174696E6700E7050164FA007E042C0128002C015E019001C8003268
S1237EC000502858021E006400190A64002C0190011E00B00496000520038A02F4010801EB
S1237EE0C800140A0601015802140A0A0A179F023D00C01C41F4012828E203D703C903B66C
S1237F0003A003840363033C030F03DE02A902720239020002C9019501640138010F01EC43
S1237F2000CC00B100990084007200630056004B004100390032002B00260022001E001AD6
S1237F400017001500120064000000640000002500250025002500250028002800280028BE
S1237F6000280001020408100810204080E2041B5B481B5B324A000D0A0020202020202051
S1237F802020206F12833A0000803F00E04D5254656368004C616D6264610054657374009C
S1197FA020202020202020202020202020202020202000401454DF
S50303FEFB
